:020000040800F2
:100000000090002019310008E92C0008ED2C0008B0
:1000100000000000000000000000000000000000E0
:10002000000000000000000000000000F12C0008AB
:100030000000000000000000F52C0008F92C00086A
:1000400069310008000000006931000869310008CA
:100050006931000869310008693100086931000818
:1000600000000000052D0008152D00082D2D0008AA
:10007000693100086931000869310008000000009A
:1000800069310008693100086931000869310008E8
:1000900069310008693100086931000869310008D8
:1000A000693100086931000869310008452D0008F0
:0800B00069310008AD2D0008C4
:1000B80010B5064C2378002B07D1054B002B02D036
:1000C800044800E000BF0123237010BD7000002029
:1000D80000000000E8810008044B10B5002B03D095
:1000E8000349044800E000BF10BDC04600000000FE
:1000F80074000020E8810008002243088B4274D372
:1001080003098B425FD3030A8B4244D3030B8B4210
:1001180028D3030C8B420DD3FF22090212BA030C19
:100128008B4202D31212090265D0030B8B4219D3FA
:1001380000E0090AC30B8B4201D3CB03C01A52411A
:10014800830B8B4201D38B03C01A5241430B8B4262
:1001580001D34B03C01A5241030B8B4201D30B034B
:10016800C01A5241C30A8B4201D3CB02C01A524172
:10017800830A8B4201D38B02C01A5241430A8B4235
:1001880001D34B02C01A5241030A8B4201D30B021E
:10019800C01A5241CDD2C3098B4201D3CB01C01A38
:1001A800524183098B4201D38B01C01A5241430942
:1001B8008B4201D34B01C01A524103098B4201D330
:1001C8000B01C01A5241C3088B4201D3CB00C01A9D
:1001D800524183088B4201D38B00C01A5241430815
:1001E8008B4201D34B00C01A5241411A00D201463A
:1001F800524110467047FFE701B5002000F0F0F8C3
:1002080002BDC0460029F7D076E7704703460B4386
:100218007FD4002243088B4274D303098B425FD3F7
:10022800030A8B4244D3030B8B4228D3030C8B4223
:100238000DD3FF22090212BA030C8B4202D3121209
:10024800090265D0030B8B4219D300E0090AC30BDE
:100258008B4201D3CB03C01A5241830B8B4201D38B
:100268008B03C01A5241430B8B4201D34B03C01A74
:100278005241030B8B4201D30B03C01A5241C30AEC
:100288008B4201D3CB02C01A5241830A8B4201D35D
:100298008B02C01A5241430A8B4201D34B02C01A47
:1002A8005241030A8B4201D30B02C01A5241CDD2EC
:1002B800C3098B4201D3CB01C01A524183098B4237
:1002C80001D38B01C01A524143098B4201D34B0120
:1002D800C01A524103098B4201D30B01C01A524183
:1002E800C3088B4201D3CB00C01A524183088B420A
:1002F80001D38B00C01A524143088B4201D34B00F3
:10030800C01A5241411A00D2014652411046704764
:100318005DE0CA0F00D04942031000D34042534069
:1003280000229C4603098B422DD3030A8B4212D329
:10033800FC22890112BA030A8B420CD3890192115B
:100348008B4208D3890192118B4204D389013AD098
:10035800921100E08909C3098B4201D3CB01C01A6D
:10036800524183098B4201D38B01C01A5241430980
:100378008B4201D34B01C01A524103098B4201D36E
:100388000B01C01A5241C3088B4201D3CB00C01ADB
:10039800524183088B4201D38B00C01A5241D9D2F3
:1003A80043088B4201D34B00C01A5241411A00D274
:1003B8000146634652415B10104601D34042002B70
:1003C80000D54942704763465B1000D3404201B5EF
:1003D800002000F005F802BD0029F8D016E77047A4
:1003E8007047C0468446100062468C461900634632
:1003F80000E0C0461FB501F0ADFA002801D4002185
:10040800C8421FBD10B501F0EDF94042013010BDE2
:1004180010B501F09FFA002801DB002010BD012073
:1004280010BDC04610B501F095FA002801DD002086
:1004380010BD012010BDC04610B501F017FA002804
:1004480001DC002010BD012010BDC04610B501F030
:100458000DFA002801DA002010BD012010BDC046A9
:10046800F0B54F464646D64643025B0A4500C0B53E
:1004780099460F1C2D0EC60F002D00D188E0FF2DC8
:1004880000D18DE08022DB00D2041A43002391467C
:1004980098469A467F3D7C027B00640A1B0EFF0F3C
:1004A800002B68D0FF2B21D08022E400D204144313
:1004B80042467F3B5B1900215D1C0A2A2EDC7E40E8
:1004C8004246022A23DC013A012A00D9BDE002296A
:1004D8006ED001292CD100200022C005F607104358
:1004E8003043E0BCBA46B146A846F0BD2B00FF3306
:1004F800002C65D00322414611433200013588465D
:100508007A40FF350A2900DDD8E01600032140466D
:1005180001228240A620C000024220D05346022B6E
:1005280046D0032B00D1BBE051464C460129D2D01E
:100538002B007F33002B70DD620704D00F2222408E
:10054800042A00D00434220103D5634B1C402B003D
:100558008033FE2B2CDCA201520AD8B2BDE79020D2
:100568008000024227D1B938FF3810426DD03E00D2
:10057800A1468A46D2E7002C41D1012342461A43BC
:1005880090462B00424601215D1C0A2A97DDC5E7EB
:10059800002B26D104239846033B00259A467AE788
:1005A800002B18D108239846063BFF259A4672E788
:1005B800FF20002291E780220026FF20D2038CE74B
:1005C80041460222013511438846FF350A29A5DC38
:1005D80002217E4074E70C239846093BFF259A4682
:1005E80059E7180002F018F94A46431F76259A4041
:1005F80000236D42914698469A462D1A4BE72000F3
:1006080002F00AF94246431F9C402B1A763B002110
:100618005D1C0A2A00DC52E780E70122D31A1B2B53
:1006280000DD58E79E352200AC40DA40631E9C414D
:100638002243530704D00F231340042B00D0043265
:10064800530137D50120002247E7210C4A462404EC
:10065800240C2700100C1204120C4443574348433F
:1006680051433A0C09195218944203D9802149027E
:100678008C4660443F0411043F0CC9198C01671E65
:10068800BC41120C890E12180C439201144312013A
:100698000ED5012362081C40144349E73E00A146D9
:1006A80080224B46D2031A435202FF20520A14E713
:1006B8001D003DE792010020520A0EE70F29EDD1F7
:1006C80080224B46D2031342EAD01442E8D13E00BE
:1006D800FF20224301E7C046FFFFFFF7F8B5474672
:1006E800CE464E0243024500720AC40F480080B548
:1006F80094465F0A2D0E9B09000EC90FB609FF2804
:1007080024D0012251402A1A8C420FD0002A00DC42
:100718006AE1002835D1002E00D1A2E0511E012A3D
:1007280000D124E1FF2A21D00A002FE0002A00DCB2
:1007380067E100285ED0FF2D18D08021C9040E4340
:100748001B2A00DC76E02A00013332E02A00FF3A57
:100758009146002E42D08C4255D04A46002A00D1FC
:100768009CE0002D00D177E00C003300DB08002B63
:1007780000D16EE08022D20313435B02FF205B0AA4
:1007880024E0FF2DF2D08021C9040E4301211B2A49
:1007980008DC31002020D140821A96403200501ED9
:1007A800824111435B1A5A0160D407212A0019407B
:1007B80057D00F211940042900D00433590150D5CE
:1007C800501CFE2A45D09B01C0B25B0AC0051843E5
:1007D800E4072043C0BCB946B046F8BD01225140E9
:1007E8008C42BAD14A46002A10D0002D00D198E098
:1007F8000023BBE7002E34D0511E012A6ED0FF2AF9
:10080800B4D00A009CE7002A00D088E0FE206A1CC9
:10081800104200D092E0002D00D0A4E0002B00D1BF
:10082800CBE0002E00D0CAE00022DB085B025B0AA6
:10083800D0B2CBE731002020D140821A9640320056
:10084800501E82410A439B185A01AED56A1CFE2DE0
:100858004AD1FF200023B9E7FF22002B4BD10C001F
:100868003300DB08FF2A00D181E7DFE79F01BF09DA
:10087800380001F0D1FF05388740854221DC3B0074
:100888002021421B0132D3408A1A97407A1E974191
:1008980000223B43590700D08BE78FE7FE206A1CF4
:1008A800104212D1002D52D1002B7CD0002EBBD08B
:1008B8009A1B500100D48BE001240022F31A0C404B
:1008C800E8E7564B2A1A3B40E4E79F1B7A0146D4D7
:1008D800002FCDD100240020002377E79B190125A4
:1008E8000132590100D460E701214D4819405B08E5
:1008F80003400B43CEE7571E012A5AD00C00FF2AAB
:1009080033D001221B2F07DC2021C91B1A008B4082
:10091800FA40591E8B411A430500B31A43E7002DCC
:1009280023D1FF22002B9BD0511E012AD6D0FF2AAB
:100938001BD01B292CDD0200731C3AE7FF2A88D044
:100948009B195B08590700D033E7DB086EE7002BDB
:1009580010D1002E43D0012433000C4006E70124B7
:10096800F71A0C4084E7002B04D13300FEE601257A
:100978009B1B18E7002E00D1F8E68022D20397428D
:1009880004D3944502D2012433000C40DB08F1E67D
:100998001A002025CA40691A8B40591E8B411343FF
:1009A80005009B1950E7002E94D0012433000C4019
:1009B8003AE70C000125F31AF5E6330034E79B19F2
:1009C80000225901C1D5154A1340DB0801222DE741
:1009D800002A00D17EE713000022DB0826E78023E7
:1009E8000024FF20DB03F1E6002A00D156E7471B6D
:1009F8003A00002D00D130E78022D2040C001343C6
:100A08007FE7002A00D101E7411B002D01D10A0030
:100A180088E78022D20413438BE7C046FFFFFFFB21
:100A2800FFFFFF7D41024200C30F490A0020120E5A
:100A38007E2A03DD9D2A02DD094A98187047802026
:100A480000040143952A07DC9620821AD1404842C7
:100A5800002BF3D10800F1E7963A9140F7E7C0463A
:100A6800FFFFFF7F70B5041E0ED001F0D5FE9E2358
:100A780001001B1A962B0CDC08282FD008398C4053
:100A88006402640AD8B201E000200024C0052043B3
:100A980070BD992B16DC421F052800D09440220017
:100AA80010480240650709D00F252C40042C05D0BA
:100AB8000432540102D59F2302405B1A9201540A62
:100AC800D8B2E3E7020020001B3290400200501E1B
:100AD80082410520401AC4401443E0E7640296208E
:100AE800640AD3E7FFFFFFFBF0B557464E4645467D
:100AF800DE46E0B583B0009001910C034F00CE0FA5
:100B0800610A009C1D03640F0C4300990092019335
:100B1800C80059004B0D9946009A019B6D0AD90FE0
:100B2800530F2B439A46009B7F0DDA0094464A46A2
:100B3800B046BA1A8E4200D1B0E0002A00DC78E054
:100B48004946002900D1E9E0C9498F4200D195E121
:100B58000125382A16DC8021534609040B439A469E
:100B68001F2A00DDE7E1202155468B1A61469D408A
:100B7800D1400D43614699404B1E99415346D3409D
:100B88000D43E41A451BA84280414042241A23021F
:100B980000D40FE16402640A002C00D139E120007E
:100BA80001F03AFE0300083B20212800CA1AD04071
:100BB8009C4002009D4022439F4200DD73E1D81B08
:100BC8000130091A2C008D40C4406B1E9D41130052
:100BD800C2408B402543002714001D436B0709D0F2
:100BE8000F232B40042B05D02B1DAB42AD416D428A
:100BF80064191D00230200D42DE19D4A0137974254
:100C080000D1D3E046469B49ED0821404A072A43D4
:100C18007C054D022D0B640D24052C43F607344347
:100C28001000210003B0F0BCBB46B246A946A0465E
:100C3800F0BD002A00D184E04A46D21B002F00D024
:100C48006DE12500054300D127E1561E012A00D198
:100C58003BE2874DAA4200D16AE20125382E12DC18
:100C680032001F2A00DDF8E120262500B61A070009
:100C78005346B040D440B540D740461EB0411B1B38
:100C88009A463D4305436246551BAC45924153463F
:100C980052420E004F4688469C1A78E7002A00DC2C
:100CA8008EE04946002975D161465346194300D163
:100CB800F6E0511E012A00D191E16D4DAA4200D102
:100CC800DCE00125382914DC0A001F2A00DDA2E136
:100CD80020215346891A8B401D006346D3401D438B
:100CE80063468B4019004B1E99415346D3400D4330
:100CF800E4182D188542804140422418230259D512
:100D08005B4B01379F4251D001215A4B6A081C4066
:100D180029400A43E507154364085FE761465346DF
:100D2800194300D1BCE0511E012A00D164E1504DA5
:100D3800AA4200D16AE10125382900DD22E70A002C
:100D48000EE74D4A7D1C154200D0D0E025006246D2
:100D5800534605431A43002F00D037E1002D00D138
:100D6800A8E1002A00D16AE16346C51A5346E21A8F
:100D7800A8429B415B42D31A1A0200D403E263469D
:100D88001D1AAC459241534652421C1B0E00884620
:100D9800A41A23E736498F4270D00125382AA8DCE7
:100DA8008021534609040B439A468EE73C000025F0
:100DB800002231E707232B40002B00D010E793E0F7
:100DC800002A74D04A46D21B002F00D1C7E0284918
:100DD800894500D185E10125382A12DC80210904E2
:100DE8000C431F2A00DDABE120212500891A0700EA
:100DF80088408D40D740411E8841D4403D4305433B
:100E0800A2446544654592415242524414004F46FB
:100E180074E7280001F000FD030018331F2B00DCE5
:100E2800C2E62A00083882409F4200DDA9E0DB1BA9
:100E3800581C1F2800DCACE115001F3BDD402028B2
:100E480005D040231B1A9A40531E9A411543072385
:100E580000272B40B0E7ED08054B62072A43E4085A
:100E68009F420FD02403250B7C05640DD4E6C046B1
:100E7800FF070000FFFF7FFFFE070000C0086207B2
:100E88000243E4081300234300D186E180252D03A3
:100E980025432D03C34C2D0BBEE6604654460E0079
:100EA8001700C508D8E7C04CFF1A144096E6BF4A99
:100EB800791C11426BD122000243002F00D0DBE0E5
:100EC800002A00D12DE1624653461A4300D1B6E00C
:100ED8006346C51885428041544440422418230281
:100EE80002D50F00B04B1C403A002800D8E76246F4
:100EF800851AA8429241534652429146E31A1A0073
:100F08004B46D21A130091461A0254D44A464C460C
:100F18002A4300D040E60026002400257CE6A14DA7
:100F2800A94500D190E00125382A00DDABE68025EF
:100F38002D042C4395E6110055462039CD40A9468D
:100F4800202A06D0402153468A1A934062461A4303
:100F5800944665466B1E9D414B461D4312E6210093
:100F6800014300D1C4E0511E012A00D1FBE08D4DA0
:100F7800AA4200D1B5E00125382900DD41E70A0081
:100F88002FE7894CFF1A14406207E4086AE7854A8C
:100F9800914200D1E3E06346C218824280412300B7
:100FA800404253441B18DD075C08072352081543C9
:100FB8000F002B4000E763461D1AAC45924153468B
:100FC80052421C1B0E008846A41AE5E5002D00D0ED
:100FD80091E0002A38D180240026240356E763468E
:100FE800C5188542804154444042241801272302F1
:100FF80000D4DFE6022787E66346C51AA842804187
:1010080053464042E41A0127241AC0E56207C00883
:101018000243E40836E7110053462039CB4099468D
:10102800202A06D0402153468A1A934062461A4322
:10103800944665466B1E9D414B461D4359E6620723
:10104800C0080243E4080DE753465A076346D80828
:1010580053460E000243DC0814E715002600203D25
:10106800EE40202A03D04025AA1A94402043421E6D
:1010780090410500354306E6002A7CD06246534677
:10108800C0081A4300D1FAE6620710438022E40838
:101098001203144208D0D908114205D16346D80872
:1010A80053460C005B071843420FC000C0085207A4
:1010B8000243E7E6002A00D12DE76346D8085346E5
:1010C8005A070E000243DC08CCE663461D1AAC45FD
:1010D8009241534652421C1B0E008846A41A0137FF
:1010E80055E56346D90853465A070A43DC08C9E65A
:1010F80060465446D4E6C008002A00D1BFE662071D
:1011080010438022E40812031442CDD0DD081542B2
:10111800CAD16346D80853465B070E002C00184313
:10112800C2E76346D90853465A070A43DC0899E6DA
:101138006346D80853465A070E000243DC08A1E666
:10114800110027002039CF40202A03D040218A1AD5
:1011580094402043421E904105003D4351E60C0057
:101168000025002258E560446045924154445242AB
:101178000500A4183AE753465A076346D908534668
:101188000A43DC087EE61A001C002A4300D0ABE6BE
:10119800C1E620210025091A19E500220025014C85
:1011A8003AE5C046FF070000FFFF7FFFFE0700008B
:1011B800F0B5DE46454657464E46E0B587B0009244
:1011C80001930B031B0B9B46CA0F4B000400804680
:1011D8005B0D029200D16AE1D44A934200D18CE1BE
:1011E8005946420FC9000A43802109041143C2002D
:1011F8009046CF4A894692469A4400230024039396
:10120800009E019F3B031B0B9B467B0030005B0D40
:10121800FD0F002B00D128E1C44A934200D177E1A9
:101228005946720FC9000A438021090411438B46AD
:10123800BF49F2008C4651466344CB1A9A460023B4
:10124800029E6E400F2C27D8BA49A40009598F4630
:10125800CB464246029E039B022B16D0032B00D19D
:10126800A6E2012B00D0DFE00022002300249046F4
:101278001B052343F60733434046190007B0F0BC6B
:10128800BB46B246A946A046F0BD002200249046BF
:10129800A64BEDE72E00DFE7CB4500D2D4E100D125
:1012A800CFE101235B429C46444648460027E2447E
:1012B8005B46150E1B021D43190C2B0412020095E8
:1012C8001D0C914602910395FEF79CFF02006A43AC
:1012D8000B04210C804619438A4209D9009D012339
:1012E800AC465B4261449C46E0448D4200D8FBE139
:1012F800881A0299FEF786FF039A240442430904D8
:10130800240C03000C43A24206D90099013B8C46E9
:101318006444A14200D8E1E1A01A424612041A43EB
:1013280093464B4659461B0C1D0004930B04494633
:101338000904090C0C001B0C5C43120C6B43884617
:1013480051436A43250CAC465B186344994203D960
:10135800802149028C466244190C24041B04240C85
:101368008A181C19904202D316D1A74214D25B46A0
:10137800009D013B4F4405934F459B41AC465B4262
:101388006344C018854200D3A1E1824200D9F6E146
:1013980000D1F1E1059B9B463C1BA742BF41009D44
:1013A800801A7F42C01B854200D1D0E10299FEF726
:1013B80029FF039A0B044243210C070019438A4270
:1013C80000D978E1881A0299FEF71CFF039A2404D1
:1013D80042430904240C03000C43A24200D95DE1F6
:1013E8004146A41A3A041A43049D13041B0C59439A
:1013F80047466B439C46100C47430B0CBC44634464
:1014080068439F4203D980256D02AC4660441F0C97
:1014180009041B04090C3F185B18BC4200D202E106
:1014280000D1FDE001231A43434B5344002B00DC59
:10143800AEE0510700D098E15946C90106D5594692
:101448003E4B194080238B46DB0053443C498B427A
:1014580000DD1AE75946D208490711435A465B0589
:1014680054028846240B5B0D02E75A46009B1A4338
:1014780000D17EE05B46002B00D100E1584601F028
:10148800CBF9020003000B3A1D27009EBA1A190077
:101498005846D64008398840320002439346009A9D
:1014A8008A40284953448A469A440023C8E65B4642
:1014B8000343994656D05B46002B00D1CDE05846F1
:1014C80001F0AAF90B235B429C460200844466465D
:1014D8001D239B1B260011005846DE400839884012
:1014E80033000343994623008B409846164B00244B
:1014F8009B1A9A460023039382E65A460243914672
:101508002AD100229A46022390460824039377E6BC
:101518005A46009B1A430D4B9C46E244002A17D1B9
:1015280002231C4300239B46023389E6FF07000081
:1015380001FCFFFF00820008FF030000FFFFFFFE21
:10154800FE070000F30300000DFCFFFF01F8FFFF9A
:10155800032332001C4373E69A460323D9460C241E
:1015680003934DE6002398469A46013304240393D7
:1015780046E601231C4300239B46013360E6002313
:10158800802498460026924B240371E60122524299
:101598000121C91A382900DD66E61F2900DCABE005
:1015A8001F204042C31A5846D8400300202904D0BF
:1015B80058468849514488400243511E8A411A437B
:1015C800072319000024114013420CD00F231340A5
:1015D800042B00D1F9E0111D91429B410A005B42A6
:1015E80059075B021C0BD2080A43904600233FE6CA
:1015F80080244B462403234209D05B46234206D16C
:101608001C4324032E009046714B240B30E68024A3
:101618004B4624031C432403029E6D4B240B27E6F0
:10162800002B00D100E70098511E84466444844290
:1016380000D284E0BC4200D2AEE000D1C1E00A0092
:10164800F0E6424500D92CE64B46DC0758084346ED
:101658005B081C434346DF072AE601F0DDF8152343
:101668009C4684440200634620321C2B00DC2EE793
:1016780023000838834099460023984636E701F04E
:10168800CBF802000300153220331C2A00DCFBE6ED
:1016980000990838814000228B4602E70099013BF7
:1016A8008C466444A14200D99AE6A24200D897E643
:1016B800831E644494E6AC466144013F8D4200D9E0
:1016C80080E68A4200D87DE6871E61447AE6854234
:1016D80000D05FE6B94500D95CE656E6A24200D8DC
:1016E8001AE6831E644417E68A4200D800E6AC4630
:1016F800831E98466144FBE53748140050448240F5
:101708005B4617008340CC407A1E974123433B43F6
:101718001A005B46CB40510709D00F21114004291C
:1017280005D0111D9142924152429B180A0019029C
:1017380000D455E7002201230024904698E50A00CA
:10174800BC4200D06EE64B4500D06BE66CE6234BFE
:10175800234A5344924500DA18E7012149420A1DF9
:101768008A42894149428B4466E60F211140042987
:1017780000D161E61100F2E7BC4200D80AE6022374
:101788005B429C4600994F444F459B41E3448C463D
:101798005B426344C018FFE54946009D4800484540
:1017A8008941AC46494261448146023A6418C7E718
:1017B80080245B4624031C4324039046044B240BDB
:1017C80056E59945E8D30A00BDE7002308E7C04677
:1017D800FF0700003E0400001E040000FF03000095
:1017E80002FCFFFFF0B55746DE464E464546E0B5DB
:1017F8000D000400E80F83460903D80F090B824641
:1018080019488C461F0369005E00490D3F0B760D91
:10181800814218D086420FD00120B1420DD1BC457B
:101828000BD1944209D1D3451CD0002905D160467B
:101838002043431E984100E00120F0BCBB46B2465D
:10184800A946A046F0BD01208E42F6D16146394333
:101858000F0017432743F0D15B465246981A431EA0
:101868009841EAE70020E8E7FF070000F0B557468F
:101878004E464546DE46E0B50D000F03390B83B0F2
:101888000400804601915800E90F314F400D8C4605
:101898006E00190382469146760D090BD80FBE4299
:1018A8001FD0BA450FD0002E2FD15546019E344384
:1018B800002D27D10A433AD0002C45D100281AD14F
:1018C8000120404217E011433BD1002E02D1019F75
:1018D8002743F3D0844509D16346002BF0D06046F6
:1018E80009E0019F27432CD1B24524D0634602204A
:1018F800013B1840013803B0F0BCBB46B246A946CC
:10190800A046F0BD002CD9D0E4E75446002CEDD019
:101918008445EBD15645E9DCDEDB019B8B42E5D8FB
:10192800DAD1C845E2D80020C845E4D2D4E700207F
:10193800002CE0D0DAE7114303D18445D6D100204A
:10194800D9E702204042D6E78445E6D0CEE7C04634
:10195800FF070000F0B557464E464546DE46E0B55F
:101968000D000F0304008046E80F390B844683B04E
:101978005800304F400D01911E0369008246914680
:10198800490D360BD80FB94220D0BA450FD00029DF
:101998002BD101990C435146002937D1324338D015
:1019A800002C44D1002819D10120404216E01643EA
:1019B80013D1002902D1019F2743F3D0844520D0B9
:1019C80063460220013B1840013807E0019F274386
:1019D80003D18A45F4D116431FD0022003B0F0BCCE
:1019E800BB46B246A946A046F0BD5446002CE7D0F7
:1019F8008445E5D15145E3DC03DB019BB342DFD8E5
:101A08000FD06346002BCFD06046E7E7002CC9D043
:101A1800D4E70020002CE1D0D2E78445D0D10020C3
:101A2800DCE7C845CCD80020C845D7D2E9E78445CB
:101A3800E3D0C5E7FF070000F0B55746DE464E463F
:101A48004546E0B51F000B031B0B16009A46CA0F4C
:101A58004B000400934687B05B0D00D1D5E0BB4A2C
:101A6800934200D1F8E05146420FC9000A43802151
:101A780009041143C2009146B54A8A469D180023BD
:101A8800984602933C037B00FA0F3000240B5B0D51
:101A9800009200D196E0AD4A934231D0720FE40033
:101AA8002243802424041443A94AF0009446634442
:101AB8005B195A1C0192424600260A2A42DC5A4601
:101AC80000994A4093464246022A32DC013A012AEA
:101AD80000D949E1022E00D1CAE0012E3DD10023F0
:101AE8000024002210005A461B052343D207134343
:101AF800190007B0F0BCBB46B246A946A046F0BDE7
:101B0800924B2643EB18002E00D1BBE0032241463E
:101B180011435A46884600994A40802109018C465B
:101B280029006144019141460A2900DD33E29346C8
:101B38000326424601279740A6213A00C9000A40D9
:101B48000F4231D0029E022E00D135E2032E00D181
:101B5800D2E154464846012EC1D0019A7D4B9446A5
:101B68006344002B00DCC0E0420709D00F2202408A
:101B7800042A05D0021D82428041404224181000E8
:101B8800E20106D5744B019A1C4080239446DB0081
:101B98006344724A93426BDC6207C00864025B05C7
:101BA8000243240B5B0D9DE7902189000F4263D10E
:101BB80088223A4200D1D7E0009BA2469B46814644
:101BC8000296BFE72300334300D17FE0002C00D109
:101BD800ADE1200000F020FE020003000B3A1D20BA
:101BE8001900821A30000839D0408C400443300074
:101BF80088405B4AEB1A944663445A1C0192424659
:101C080000260A2A00DC5AE79CE753460343994614
:101C180054D05346002B00D177E1504600F0FCFD2C
:101C28000B235B429C46020084441100504608394D
:101C380088401D23804660461B1A2000D8400300B8
:101C4800404603439A4623008B4099460023444D5F
:101C58009846AD1A029315E752460243914626D19B
:101C680000221D000223924608329046029309E79B
:101C780000240022354B35E7002380249B462403AB
:101C8800324B2FE70222414611438022120194462B
:101C98002A006244884601920A2900DD52E75A4622
:101CA8000020009904004A40934602260BE70C22C4
:101CB8001D000323814690460293E3E600239A46DB
:101CC80004339846033B00250293DBE64246013382
:101CD8001A432B0090465A1C0192424600240020C9
:101CE80001260A2A00DCEAE62CE70122D21A382A61
:101CF80000DDF4E61F2A00DC2AE11F214942CB1A45
:101D08002100D9400B00202A05D0164A019D94468F
:101D18006544AC402043421E9041184307231900F4
:101D28000024014003420CD00F230340042B00D1B0
:101D380040E1031D8342A441180064426107640224
:101D4800240BC20800230A43CCE6C046FF07000064
:101D580001FCFFFFFF030000FFFFFFFEFE0700007E
:101D68000DFCFFFF3E04000049464A460904090CE1
:101D78000D00160C020C0004000C4543AC4605008F
:101D88007543A84615000F007543009202952A0076
:101D9800009D6F4365462D0CA94647444F44B845FE
:101DA80005D91500802252029046454402953D0C03
:101DB800039565462D043F042D0CAC463D00654453
:101DC8000495250C2404240CAC4625007543A8462C
:101DD80065460F006943414489466743390C4944C5
:101DE8006E43884503D980225202904646440D0C22
:101DF800A846350045440595039D3F04A8463F0C79
:101E08000904C91988444546039555462E04360CDD
:101E18002F0C35004543784381463800A8462D0CE1
:101E2800AA46009A504372434A445244914503D902
:101E380080256D02A9464844150CA94645462D043F
:101E48002D0CA84665467D43120448449044A94693
:101E58003200654662436E437C43170C3619BF193E
:101E6800BC4203D980246402A446E144029C039E38
:101E7800A446059D66448E428941AC4612043C0442
:101E8800120CA2186244494254184644A4464645D6
:101E9800A44182466442A046AA4292418C458941A7
:101EA800E244D044494252420A43A045A4418245F3
:101EB8008941644249420C4341463F0CD2191219E8
:101EC800CC0D049970020843411E884141464A449A
:101ED800F60D52023043490214430843D20135D566
:101EE8000122430802401343E0071843640834E61C
:101EF800009BA2469B4681468024534624031C43EC
:101F080024034A462E4B240BECE500F085FC1523F0
:101F18009C4684440200634620321C2B00DC84E685
:101F2800002399462300083883409A468EE600F03D
:101F380073FC02000300153220331C2A00DC4EE635
:101F480002003400083A0020944052E6019304E667
:101F58001C4B21009C460300019DD3406544A940C9
:101F680019430300AB40581E834119430800D4406D
:101F78004B0709D00F230B40042B05D00B1D8B42B8
:101F88008041404224181800230200D4D6E60123D9
:101F980000240022A6E50F29AAD1802352461B035C
:101FA8001A42A9D01C42A7D11C43009B02009B46A1
:101FB800034B97E50024C1E60024014B220091E57C
:101FC800FF0700001E040000F0B54E464546DE46F9
:101FD8005746E0B585B0009001910C034F00CE0F35
:101FE800610A009CB046640F0C4300997F0DC8003D
:101FF80011001A001B039C460091019251004B0DE1
:102008009946019B009DD90F63466A0F5B0A1343EB
:10201800EA0094469346C14A03900293914500D141
:10202800CDE0012569404D467D1BAA468E4200D170
:1020380080E0002D00DC35E34946002900D1DFE0CF
:10204800974200D194E152460125382A19DC8022B2
:10205800029B12041343029352461F2A00DDE3E158
:10206800534620226146029DD21A9540D9400D431D
:10207800614691400A00511E8A411543029ADA408E
:10208800A41A451BA84280414042241A230200D4C6
:102098003DE16402640A002C00D147E1200000F011
:1020A800BBFB0300083B20212800CA1AD0409C40F3
:1020B80002009D4022439F4200DD77E1D81B01309A
:1020C800091A2C008D40C4406B1E9D411300C2406C
:1020D8008B402543002714001D436B0709D00F23AD
:1020E8002B40042B05D02B1DAB42AD416D4264192A
:1020F8001D00230200D440E1884A0137974200D1ED
:1021080001E1012643468649ED0821404A072A4352
:102118007C054D022D0B640D1E4024052C43F6074B
:1021280034431000210005B0F0BCBB46B246A946B6
:10213800A046F0BD002D00DCD0E24946002900D0C1
:10214800D4E06146029B194300D12BE1691E012DA1
:1021580000D1D9E1954200D10AE10125382917DCDF
:102168008A4653461F2B00DDE7E12022D21A029B44
:10217800614693401D005346D940634693401A0078
:102188000D43511E8A4153461543029ADA40A4185A
:102198002D188542804140422418230200D4B6E01D
:1021A8005E4B01379F4200D1ADE001215C4B6A08CC
:1021B8001C4029400A43E507154364088DE7594A3E
:1021C800029B92466246BA441A432CD08E422ED0C5
:1021D8005246002A60D0002F00D1DBE063460E0093
:1021E800029CD80862070243E4081300234300D185
:1021F80054E280252D0325432D03484C2D0B8CE7F5
:102208006146029B194300D1CCE029000139012D18
:1022180000D188E1954200D1AAE00125382900DDE6
:102228002FE78A4618E7012251408E42D0D1534603
:10223800002B00D1BEE0002F00D038E1CA462200B2
:10224800024300D1E2E15346591E012B00D10DE2B1
:10225800324A924500D1D2E10127382913DC1F29DF
:1022680000DDEEE12022029B521A250007009A4663
:10227800CC4090409540CF40A244421E90415346E6
:102288002F43074302933D00654465459241029BF5
:1022980052424F46D41880E7234A7D1C154200D08D
:1022A800AAE062462500029B05431A43002F00D08E
:1022B800F5E0002D00D16BE1002A00D152E1634620
:1022C800C51A029BE21AA8429B415B42D31A1A0222
:1022D80000D4D5E163461D1AAC4592410126029B04
:1022E80052421C1B8846A41A0E40F6E697423FD07D
:1022F80052460125382A00DD4AE78022029B120453
:10230800134302932DE73C000025002205E707232D
:102318002B40002B00D0E2E66BE0C046FF07000030
:10232800FFFF7FFF01F8FFFFFE070000280000F015
:1023380073FA030018331F2B00DCB4E62A000838B0
:1023480082409F4200DDB9E0DB1B581C1F2800DCDF
:10235800A0E115001F3BDD40202805D040231B1AB3
:102368009A40531E9A411543072300272B40D0E774
:10237800C00862070243E40837E7EA0863071A431C
:10238800D34BE4089F4200D12FE72403250B7C059B
:10239800640DC2E6CA462200024358D163460E00C5
:1023A800029C0393039B5746DA08E7E7C94CFF1AD8
:1023B800144092E6C84D7A1C2A4200D084E02200DC
:1023C8000243002F00D0EFE0002A00D1E5E062468A
:1023D80002990A4300D1C5E06346C5188C46854278
:1023E8008041644440422418230202D5B94B013786
:1023F8001C40BA460395D5E76246851AA842924121
:1024080052429146029BE31A1A004B46D21A130015
:1024180091461A026CD44A464C462A4300D03AE602
:1024280000260024002578E6029953460D00203A3C
:10243800D540202B06D04022D21A0B00934062468A
:102448001A4393465B465A1E93411D4319E6534669
:102458005A1E012B00D1C6E09D4EB24500D1BDE603
:1024680088460E000125382A10DC1F2A7FDC20212F
:102478002500891A070088408D40D740D440411E66
:102488008841029B3D431B1B054302936246551B33
:10249800AC459241029B52424F469C1AF6E5002DEC
:1024A80000D0B7E0002A00D1F0E001260E406346D4
:1024B8000298D90842070A43C40896E6854CFF1AD1
:1024C80014406207E40860E781498A4200D1C9E004
:1024D8006346C11881428041029B4042E3181B18A1
:1024E800DD075C08072349080D4317002B4010E758
:1024F80063461D1AAC4592410126029B52421C1BA1
:102508008846A41A0E40C6E56346C518029B854254
:1025180080419C464042644424180127230200D489
:10252800F5E6022741E66346C51AA8428041029BA8
:102538004042E41A0127241AA8E5029D52462B00BE
:10254800203AD34019005346202B06D04022D21AF5
:102558002B00934062461A4393465D466B1E9D418D
:102568000D4315E66207C0080243E4080DE71100B1
:1025780027002039CF40202A05D040218A1A9440CC
:10258800250005430395039D6A1E95413D437DE75C
:10259800002A00D144E701260E406346D908029B71
:1025A8005A070A43DC08F0E6002A28D06246029F50
:1025B800C0083A4300D1DCE6620710438022E408F1
:1025C8001203144209D0FD08154206D163460126BC
:1025D8002C00D8087B0718430E40420FC000C008E3
:1025E8005207024301E663461D1AAC459241029B1D
:1025F80052421C1B0E0088460127A41A46E5634672
:10260800D908029B5A070A43DC08EEE56346029C98
:102618000393C7E6C008002A00D1AAE66207104360
:102628008022E40812031442D7D0029FFD08154205
:10263800D3D163460126D8087B072C0018430E40E7
:10264800CBE70A002700203AD740202905D04022AE
:10265800521A9440250005430395039D6A1E95412F
:102668002F4310E614000025002256E5029B604423
:102678009946604592414C4452420500A4184CE7E3
:102688001A001C002A4300D0B3E6C9E680240026BD
:102698002403AEE520210025091A17E500220025AC
:1026A8000B4C3AE5002D00D1F6E54B46DA1B924675
:1026B800002F00D16FE6382A05DC80263604344323
:1026C80088460E00D1E688460E000125DEE6C046A3
:1026D800FF070000FFFF7FFFFE070000002D00D16D
:1026E80068E64B46D91B002F01D18A46A7E501278A
:1026F800382900DDC7E5802212041443AFE5C0463F
:10270800F0B5C6461E03360BB0460D4E0C034D0001
:102718005F0000B5240B6D0D7F0DB5420BD0084945
:1027280000208F4204D1464616433000431E98418C
:1027380080BCB846F0BD04430120002CF8D1EEE778
:10274800FF0700000B00020070B5164D0C0382B0A5
:102758004900002000920193240B490DDE0FA94285
:1027680004DD1148814203DD104BF01802B070BD42
:102778008020400320430E4C641A1F2C08DD0D4BAB
:102788005B1AD84003005842002EEFD11800EDE73D
:10279800094B009A9C46030061448B40E240134376
:1027A800F1E7C046FE0300001D040000FFFFFF7FA5
:1027B8003304000013040000EDFBFFFF70B5002890
:1027C80016D0C317C5185D40C40F280000F024F8C0
:1027D800104B1B1A5B055B0D0A2814DC02002E0047
:1027E800153296400B22121AD5402D032D0B03E00B
:1027F80000240023002500261B052B43E407234360
:102808003000190070BD0B3885402D0300262D0BB4
:10281800F2E7C0461E0400001C2101231B04984255
:1028280001D3000C10391B0A984201D3000A083959
:102838001B09984201D30009043902A2105C401810
:102848007047C046040302020101010100000000B4
:102858000000000010B584B00C22002101A805F08A
:1028680075FB8022344C354B92030521236022618D
:10287800802304225B036261E161033A27316254D9
:10288800636000210023A27606326263A2632000FF
:102898003532A360E36023836362A3622363A15498
:1028A800E36400F0C9FC002834D10123019300231C
:1028B800200001A90293039300F034FE002838D1C8
:1028C8001F4B20000193042301A9029300F02AFE64
:1028D80000282BD11B4B20000193082301A9029348
:1028E80000F020FE00281ED1174B200001930C2376
:1028F80001A9029300F016FE002811D1134B200005
:102908000193102301A9029300F00CFE002804D1C2
:1029180004B010BD00F0C6F9C7E700F0C3F9F7E747
:1029280000F0C0F9EAE700F0BDF9DDE700F0BAF918
:10293800D0E700F0B7F9C3E7E80000200024014021
:1029480002000004040000080800000C1000001039
:1029580070B504008EB01422002102A805F0F6FA22
:102968001C22002107A805F0F1FA274B22689A4299
:1029780001D00EB070BD8023DB010793802307A828
:102988001B060C9303F0F2F8002837D180211F4B67
:1029980049031A6CA0200A431A641A6C00260A40DC
:1029A8000092009A0122596BC005114359635B6B71
:1029B80002A91A400192019B1F2203230496029246
:1029C800039301F0B5F9124D124B28002B60052333
:1029D8006B607B332B6180336B618023DB00AB61E1
:1029E8002023EB6180235B01AE60EE602B6200F078
:1029F800EBFF002805D12565AC62BAE700F052F973
:102A0800C4E700F04FF9F6E7002401400010024047
:102A18008C000020080002400123124A00B5916B87
:102A280083B019439163926B0021134001930022F4
:102A38000920019B00F078FF092000F09FFF002289
:102A480000210A2000F070FF0A2000F097FF002202
:102A580000210B2000F068FF0B2000F08FFF03B06F
:102A680000BDC0460010024010B588B014220021F5
:102A780002A805F06BFA0222184B194C596B20007A
:102A880011435963596B0A400092009A0122596B0D
:102A9800114359635B6B13491A4001920122019B50
:102AA80001F038FAC0220123920002920393002217
:102AB8000123200002A90492059301F039F90222AA
:102AC80001230292039300220223200002A9049208
:102AD800059301F02DF908B010BDC0460010024062
:102AE800000400500203000010B5194B194C0122D4
:102AF8002360194B200063600023E260A360236118
:102B08006361A361E361236201F086FE00280CD1B2
:102B18000021200002F0E2FB00280ED10021200055
:102B280002F002FC002810D110BD00F0BBF8002113
:102B3800200002F0D3FB0028F0D000F0B3F8002109
:102B4800200002F0F1FB0028EED000F0ABF8EBE734
:102B5800005800404C010020BC7D701010B50400E6
:102B680088B01422002102A805F0F0F9124B22685F
:102B78009A4201D008B010BD0123104CA020626B0E
:102B880002A91A436263626BC00513400093C02216
:102B9800009B12235201029203930623069301F02D
:102BA800C7F88022E36BD2031343E363E36B13405C
:102BB8000193019BDEE7C046005800400010024028
:102BC80009480A4B10B5036003234360FA231B012D
:102BD800C360074B836002F0D5FB002800D110BD0D
:102BE80000F060F8FBE7C046A0010020003000407C
:102BF800B80B000000B593B03422002105A805F0F9
:102C0800A5F910220021684605F0A0F9802080006F
:102C180002F0F4FB0A230593F63308930023099383
:102C28000E9308330F93C0234022DB0210938023B6
:102C38000A923F3A0B929B05013205A80C920D921D
:102C4800119302F00BFC002801D072B6FEE70722B0
:102C58000223009201930022002302216846029277
:102C6800039302F0A7FE002801D072B6FEE713B066
:102C780000BDC04610B500F09BFAFFF7BBFFFFF799
:102C8800F3FEFFF7C9FEFFF7E5FDFFF72DFF00F0A4
:102C9800BFF800F0EDF800F033F9FFF791FF04F00A
:102CA8002FFFFEE772B6FEE701220C4B00B5196C48
:102CB800C02011431964196C83B00A408021009226
:102CC800009ADA6B49050A43DA63DB6BC0000B40F4
:102CD8000193019B00F0A4FA03B000BD001002406C
:102CE800FEE7C046FEE7C0467047C0467047C0468C
:102CF80010B500F071FA05F01FF810BD10B50248C4
:102D080000F0B8FF10BDC0468C00002010B5034885
:102D180000F0B0FF024800F0ADFF10BD1003002026
:102D2800B402002010B5034800F0A4FF024800F0E8
:102D3800A1FF10BD58020020FC01002070B5144C02
:102D4800200003F083FA200003F034F910222368EE
:102D5800D9690A4204D01A620E4B1A78002A06D0A2
:102D68000D4D29008022200003F0A8F870BD0B4A01
:102D7800094D12680A48516880225242521AD2B24A
:102D88001A701A782900D2B205F012F9E9E7C0469C
:102D9800000400207C0A0020FC0900201003002009
:102DA800FC08002070B5144C200003F04FFA2000F6
:102DB80003F000F910222368D9690A4204D01A6284
:102DC8000E4B1A78002A06D00D4D290080222000CB
:102DD80003F074F870BD0B4A094D12680A4851682F
:102DE80080225242521AD2B21A701A782900D2B2EC
:102DF80005F0DEF8E9E7C0466C030020F80800207B
:102E080078080020FC010020780700207047C046A1
:102E18000A480B4B10B503601423FA2243600023C1
:102E280092008360C2600361836102F069FF002839
:102E380000D110BDFFF736FFFBE7C046B001002008
:102E480000200040084B026882B09A4201D002B0CC
:102E580070478021054B09021A6C0A431A641B6CDF
:102E68000B400193019BF2E7002000400010024054
:102E780010B5214B214C0C222360E1235B026360D7
:102E880000232000A360E36023616261A361E36122
:102E980023626362A36203F0DFFD002811D10021E1
:102EA800200003F0EFFE002813D10021200003F0DA
:102EB80039FF002815D1200003F0C8FE002817D1DB
:102EC80010BDFFF7EFFE0021200003F0DBFE002815
:102ED800EBD0FFF7E7FE0021200003F023FF0028D6
:102EE800E9D0FFF7DFFE200003F0B0FE0028E7D0AE
:102EF800FFF7D8FEE4E7C046003801400004002090
:102F08000C480D4B10B50360E1235B020C224360B3
:102F1800002342618360C36003618361C36103620C
:102F28004362836203F098FD002800D110BDFFF7CB
:102F3800B9FEFBE76C0300200048004070B50400B0
:102F480090B01422002104A805F000F81C220021EA
:102F580009A804F0FBFF2368614A934204D0614A40
:102F680093425DD010B070BD012309A8099302F007
:102F7800FDFD002800D0AAE080215B4BC9011A6C36
:102F880000260A431A641A6C58480A400092009AAC
:102F98000222596B114359635B6B04A913400193D7
:102FA800019BC0230592049306960796089600F0A5
:102FB800BFFE4F4D4F4B28002B6032236B604E33C2
:102FC8002B6180239B01AE60EE606E61AE61EE61A5
:102FD8002B6200F0F9FC002876D18022464BA550E0
:102FE800AC62464D2B6033236B60233BAB60002300
:102FF800EB606B61AB61EB61802328009B012A6168
:103008002B6200F0E1FC00285BD1002200211B208C
:10301800E567AC6200F088FC1B2000F0AFFCA1E77C
:103028008021314BC902DA6B30480A43DA63DA6B24
:103038000A400292029A0222596B114359635B6B50
:1030480004A91A400392039B0522022304920593C4
:103058000423089300F06CFE294D2A4B80222B6034
:1030680037236B60273BAB6000232800EB602A61A5
:103078006B61AB61EB612B6200F0A6FC002829D1E3
:10308800214BE567AC62214D80222B6036236B60B3
:1030980000232800AB60EB602A616B61AB61EB61D8
:1030A8002B6200F091FC002817D180230022002118
:1030B8001D20E550AC6200F037FC1D2000F05EFCDE
:1030C80050E7FFF7EFFDA0E7FFF7ECFD85E7FFF717
:1030D800E9FD51E7FFF7E6FDD2E7FFF7E3FDE4E797
:1030E8000038014000480040001002400004005031
:1030F800100300201C00024030000240B4020020EF
:10310800580200204400024058000240FC01002000
:103118000D488546FFF77AFE0C480D490D4A0023F5
:1031280002E0D458C4500433C4188C42F9D30A4A74
:103138000A4C002301E013600432A242FBD304F0DE
:1031480013FFFFF797FDFEE7009000200000002026
:1031580070000020D0820008700000203C0C002085
:10316800FEE7000070B50F4B04001978002901D163
:10317800012070BDFA208000FCF7BEFF0A4D010057
:103188002868FCF7B9FF00F005FC0028F0D1032CF3
:10319800EED801380022210000F0C6FB034B0020C6
:1031A8001C60E6E704000020000000200800002062
:1031B8008023084A5B00116810B50B430320136095
:1031C800FFF7D0FF041E02D00124200010BDFFF736
:1031D8006BFDFAE700200240034A044B11681B7894
:1031E8005B1813607047C046940400200400002058
:1031F800014B18687047C0469404002070B504005D
:10320800FFF7F6FF0500631C02D0044B1B78E41897
:10321800FFF7EEFF401BA042FAD370BD0400002068
:10322800034A044913680B40034313607047C046C0
:1032380000000140FFF9FFFFF0B5D6464F4646466D
:103248000023C0B582B0041E01932CD0856D002DDB
:1032580000D1CCE0802325685B05AA681A4215D105
:10326800AA687B490A401343AB607A4B7A491868CD
:10327800FCF742FF013040000190019B002B05D074
:10328800019B013B0193019B002BF9D1AB68002006
:10329800DB0000D49DE0AB685B070BD5A36D102263
:1032A800A36D1343A365012002B0E0BCBA46B14642
:1032B800A846F0BDA36DDB06F1D4A36D674A21696A
:1032C80013400632FF321343A365AB68DB075CD4B7
:1032D800276BA2687B1E9F41E368A67E1A43237E64
:1032E8003F039B031A43637EDB031A4373031A43AA
:1032F800002900DA9BE080239B039C462C23E35C97
:103308005B0013433B43624620271343E25D012AD7
:1033180000D190E0626A002A05D0E02676003240AB
:10332800A66A324313433C27EA684D4E32401343A2
:103338006668EB60E26CE75DB30F9B079A46BC4694
:103348001A43012F09D1676C236C3B431A43534638
:10335800A76C3A431A4363461A432B69414F3B40D3
:10336800134380222B6173005B08D20593420CD073
:1033780080231B069E4208D03B4A3C4F13683B40C3
:10338800F027BF033E4033431360072670276B695D
:10339800626BB34313436B616E69A36BBE431B013E
:1033A80033436B61002928D11023A96A5B420B4380
:1033B800AB62072369690B409A422FD01222A36D92
:1033C8009343023A1343A365E36D0F3A1343E3654E
:1033D80069E71022A36D01201343A365E36D0F3A3B
:1033E8001343E365AB685B0700D463E756E7FFF771
:1033F800AFFA5423E565E5542CE780239B039942F3
:10340800D7D11C21AB6AE369013B9B00194010230B
:103418005B428B40216E0B43AB62CAE70023032259
:10342800E365A36D9343023A1343A3653CE74B005E
:103438005B089C4662E7002E03D1802252021343A8
:1034480068E7A66D3E43A665E66D3243E26561E72F
:10345800E8FFFF6F00000020400D0300FDFEFFFFA6
:103468000102DEFF02FCFF1F08270140FFFFC3FF28
:103478007047C0467047C04610B5806AFFF7FAFF2C
:1034880010BDC0467047C0464022806A10B5836DA3
:1034980013438365C36D3C3A1343C365FFF7F2FFDB
:1034A80010BDC04650210300806A10B5826D1142DC
:1034B8000DD18023826D9B001343C022836503686E
:1034C8001201D96811420AD0FFF7D2FF10BD826DF0
:1034D800D20616D4026D1800526B9047F6E7827E2A
:1034E800002AF1D11A681207EED59A6852070BD54F
:1034F8002022836D13438365C36D1F3A1343C3654D
:10350800E2E7FFF7BFFFE1E70C215A688A435A60F8
:10351800836D034A13400432FF3213438365D3E7B4
:10352800FEFEFFFFF0B5DE4657464E4645460023F1
:103538000400E0B585B003935433E25C0069012AC6
:1035480000D19AE00122E254236803329E68324295
:103558000ED00120A36D1C321343A365542300220F
:10356800E25405B0F0BCBB46B246A946A046F0BD41
:103578004E68904384460868022E5ED047037D0B50
:10358800802700953F06BC4553D0276EBB461F27B2
:10359800B8463740BA460F275546AF40FD43BC46AC
:1035A80001955F466546AF43009DB946002D66D13B
:1035B8004546820E15402A005546AA404D461543F9
:1035C800A9464A46B6082266E2690136964208D8F4
:1035D80056468200120FB2409D6A019E35402A432A
:1035E8009A6205028A6829005E692A40664D8E4300
:1035F8002A4032435A61002801DB0020AEE7E0216F
:10360800624D634A2B684904194090424CD0614A84
:10361800904240D0604A9042EFD18022D2031342B8
:10362800EBD12B685D4803400B431A4300202A6006
:1036380094E79A6A2A439A62D3E78022120694454D
:1036480004D19A6A4103490B8A439A620028D4DA62
:103658004E4A4F491368884223D04E4988424AD07F
:103668004D498842C9D1C0201168400403404B48E5
:1036780001400B430020136070E7022071E7012529
:1036880005429ED1022707422DD0524695404A4610
:103698002A43914695E7802252041342C1D0002064
:1036A8005CE7A0201168E0E7802212041342A4D14D
:1036B8002B683A4803400B431A43394B2A60186871
:1036C8003849FCF719FD013043001B189B00039390
:1036D800039B002B91D0039B013B0393039B002B7F
:1036E800F9D100203AE7024209D0524697404A46AB
:1036F8003A43914665E7C02011680004B6E702071F
:1037080001D5032258E7C20601D5042254E78206F0
:1037180001D5052250E7420601D506224CE70206EC
:1037280001D5072248E7C20501D5082244E78205EA
:1037380001D5092240E7420501D50A223CE70205E6
:1037480001D50B2238E7C20401D50C2234E78204E4
:1037580001D50D2230E7420401D50E222CE70204E0
:1037680004D55A4665462A4391462AE7C20301D53D
:10377800102221E7820301D511221DE7420300D45C
:103788001FE7122218E7C04600FFFF07082701407D
:10379800001000B0004000B8002000B4FFFF3FFE5A
:1037A80000000020400D030000230122F0B583B083
:1037B80001930368040099680A421FD19868284950
:1037C80008421ED19968274801400A439A60264B4F
:1037D8001B681B020FD5254B25491868FCF78CFC84
:1037E80001300190019B002B05D0019B013B019307
:1037F800019B002BF9D1637E012B0BD1002003B074
:10380800F0BD1021A36D01200B43A365E36D1343A5
:10381800E365F4E7FFF7ECFC236806001A68D207B3
:10382800ECD401250F4F9A68154203D19A683A40A3
:103838002A439A60FFF7DCFC2368801B022802D920
:103848001A68154203D01A681542ECD0D6E7102240
:10385800A36D01201343A365E36D2B43E365CEE716
:1038680017000080E8FFFF7F0827014000000020C4
:10387800400D0300F0B5C64605680400AE688846EA
:103888001700022000B5760714D45422A35C012B3C
:1038980010D00123A354EA68134206D1AA68134240
:1038A80031D10122EB681343EB602000FFF77CFF66
:1038B800002802D080BCB846F0BDA26D154B256D1E
:1038C8001A4080235B001343A365134BE065EB624A
:1038D800124B10222B63124B21686B631C230B6065
:1038E8003833E0544B68280013434B6042463B0092
:1038F800403100F0DFF822680A4993680B40042140
:103908000B439360D6E7AB68064A13400343AB60AA
:10391800C7E7C046FEF0FFFFAD3400088134000859
:1039280091340008E8FFFF7FFF22032310B514003D
:103938000340DB009C4089010A40E4439A40002888
:103948000BDB0C4BC0219C4680088000604489003A
:10395800435823401343435010BD0F2306490340E7
:103968008C46083B9B089B006344D9690C40144370
:10397800DC61F1E700E100E000ED00E0002805DB94
:103988001F22012302409340014A13607047C0463A
:1039980000E100E08022431E5204012093420ED22F
:1039A800C021074A07485360036A09061B021B0A1D
:1039B8000B430362002300209360073313607047B2
:1039C80010E000E000ED00E0F0B5C646040000B5E8
:1039D800002860D00568314B1421E818FCF78CFBEF
:1039E8008300236402222523E2542B682C4AA6680C
:1039F80013402B60E368216933430B4361692A68EC
:103A08000B43A1690B43E1690B43216A0B43134341
:103A18002B60244B14219C4660448700FF20224BD6
:103A28002840A364676408389846FCF765FB1F23A1
:103A380001220340100098408023E064DB019E428D
:103A48001FD03F23454661680B4001393B606860E1
:103A580003291BD8154916485918013B9A400023D9
:103A6800890021656065A2650B60426000232522FC
:103A780001210020E363A154013AA35480BCB84655
:103A8800F0BD002363603B60434658600023236514
:103A98006365A365EAE70120F0E7C046F8FFFDBFCC
:103AA8000F80FFFF00820010800802403F82001054
:103AB80040090240F0B5C646242400B5055D012D35
:103AC8004FD0012525260555855DEFB2012D07D07C
:103AD8008023C36300230355012080BCB846F0BD92
:103AE800223C84550024C4630468C66C2568BD4321
:103AF8002560856C6E60066D002E02D0456D876D61
:103B08006F601F4D076CAC466D68A8461C252F409A
:103B18001B3DBD4047463D4367467D606360836803
:103B2800102B20D0A160E260036B002B1ED00E2268
:103B3800236813432360426C1368DB0304D5802396
:103B480011685B000B431360002E04D08023326899
:103B58005B00134333600122236800201343236072
:103B6800BBE70220B9E7A260E160DDE70422236831
:103B7800934323602368063213432360DBE7C04680
:103B88000000024070B5002832D02523C35C022B08
:103B980029D10E210268174C13681C268B43416CEF
:103BA80013600B6823400B6001231168994311606F
:103BB800026C1149324093404D682B434B60C26CF4
:103BC800836C5A60036D002B05D01A6822401A6076
:103BD800436D826D5A6025230122C2540022013BA5
:103BE800C254002070BD04230022C3632033C25492
:103BF8000120F7E7FFFEFFFF00000240252370B514
:103C0800C35C022B03D00423C363012070BD0E21C3
:103C180002681C261368154C8B4313600123116836
:103C280099431160416C0A6822400A60026C10498D
:103C3800324093404D682B434B60C26C836C5A6092
:103C4800036D002B05D01A6822401A60436D826DFF
:103C58005A6025230122C2540022013BC254836BBF
:103C6800002B00D098470020D0E7C046FFFEFFFF9A
:103C78000000024070B51C2104242B4B06681A680A
:103C8800036C35680B40210099400A4210D02C4241
:103C98000ED033689B0602D43368A3433360224BAB
:103CA8005A6811435960036B002B00D0984770BDC8
:103CB8000224210099400A4217D02C4215D03368BB
:103CC8009B0606D40A223368934333602523093AB6
:103CD800C254154B5A681143596000222423C25418
:103CE800C36A002BE3D09847E1E708210C009C4009
:103CF8002242DCD02942DAD0326806318A43326067
:103D0800012215009D402B0007494C6823434B6056
:103D18002523C263C2540022013BC254436B002BCB
:103D2800C5D09847C3E7C04600000240C06B704743
:103D3800F0B5DE4657464E464546E0B50C688B461C
:103D4800002383B0002C68D001229A409446224078
:103D58009246624614425CD003215A465F00B9403D
:103D680055680322C9432A40561E0091012E5BD98B
:103D7800032A00D0ADE0BA400668009931400A43F2
:103D88000260C0229202154243D003270F265D49E4
:103D98001F408C46FF00BE409A0892006244116E94
:103DA800B143A026F605B0420ED0574EB04200D11E
:103DB800A0E0564EB04200D1A0E0554EB04200D12E
:103DC80094E00526BE4031438026116651464D4A8F
:103DD8007603C9431268354200D077E00A40494E5D
:103DE800326072688026B60335426CD10A40454E6F
:103DF80072608422B258AF0362D40A408427414ECD
:103E0800F2518022B258ED0356D40A4080213D4D2C
:103E18006A5022000133DA4096D103B0F0BCBB46A9
:103E2800B246A946A046F0BD81680E0000990E4032
:103E38005946C968B1460E00BE40B0464E46414696
:103E48000E43866041680E0061468E432909B046DC
:103E58000E0001210E409E40B446464661460E4380
:103E68004660C1680E0000990E4059468968B04600
:103E78000E00BE40B446464661460E43C660022A5E
:103E880000D078E7D90889008C46844461460E6AD8
:103E9800072119408900884601960F214646B140FE
:103EA800019E8E435946019646460969B140019ED6
:103EB8000E4361460E625EE7514611430A00A5E7CC
:103EC800564632439AE75646324390E756463243BF
:103ED80085E70E00C1683140884659468968B9406F
:103EE8008C46414666463143C16044E70326BE40DE
:103EF800314369E70126BE40314365E70226BE40EB
:103F0800314361E7001802400004005000080050E7
:103F1800000C0050002A01D0816170478162FCE7E3
:103F2800426913000B401B0491430B4383617047A4
:103F3800F0B557464546DE464E46E0B583B001919A
:103F48001021036888469A69323104008A461204AF
:103F580000D496E042464046996900250A40084246
:103F680041D0002293468022120200279146019EEA
:103F7800D86120359A6915422DD1002F2ED1FFF72F
:103F880037F92368801B1928F4D952465868A25C6F
:103F98009969D2B294464A4611420DD08021C9018E
:103FA800084209D16246202A06D05A68114359604E
:103FB800FFF71EF9060023689A691542DAD1FFF760
:103FC80017F92368801B1928F6D9202293469A6985
:103FD80001271542D1D0002F00D1DD6104225946B6
:103FE80011430A000125802099694000014234D01C
:103FF8000125D8612A43480504D5082002438020BA
:10400800C000D861890504D502210A43FF31FF3178
:10401800D9619969890701D50021996201219869B7
:10402800014202D198690143996159681A480140CF
:104038005960636C1343636420224123E2540022D5
:104048000133E254402300220120E25403B0F0BCC3
:10405800BB46B246A946A046F0BD4805CDD4890561
:10406800D2D4002DD5D1FFF7C3F8019BC01A23681D
:10407800192802D99A69120405D49A69120400D53C
:1040880068E70020E2E72022636C1343636441235E
:10409800E2540133E554D5E700E800FEF0B5574691
:1040A8004E46DE4645461024E0B506000F0083B0B4
:1040B800036801920225B3462A0099690A400D4215
:1040C80000D072E0210098690026014004420BD01C
:1040D800DC61791C6DD1202099690842FCD020212F
:1040E800D96104210126114380209A6940000242C7
:1040F80035D001245E462143D861500504D50820F7
:1041080001438020C000D861920504D502221143E2
:10411800FF32FF32DA619A69920701D500229A626A
:1041280001229869024202D1986902439A615A6849
:10413800514802405A60736C20220B437364412338
:10414800F25400220133F254402300220120F25499
:1041580003B0F0BCBB46B246A946A046F0BD500528
:1041680001D55E46CBE7920501D55E46CEE7002E27
:104178001DD17A1CA0D0FFF73BF85E46019BC01A00
:104188003368B84201D8002F94D1022108009A69F7
:104198001040114200D08DE72022736C13437364E2
:1041A8004123F2540133F054CEE70020D0E75E46B5
:1041B800B1E701990092884600213A0089464231C8
:1041C8005F4620268A4693469A6916420FD14A4688
:1041D800002A4BD1FFF70CF84346C01A83450FD38A
:1041E8005B46002B0CD03B689A691642EFD05946C3
:1041F800BB460F004946009A002900D16FE770E7D7
:1042080052463B685868BA5C9969D2B29446802293
:10421800120211421ED08021C90108421AD16246F9
:10422800202A17D05A6811435960FEF7E1FF3A0077
:104238003B689046070006E0FEF7DAFF4346C01BDE
:1042480019280BD81B689A691642F5D04246B84619
:104258001700B9E73A0047469046F4E72022009253
:104268001F3AB84691461F001B68ADE75946009AA9
:10427800BB460F0035E7C04600E800FEF0B55746DC
:10428800DE4645464E461024E0B5924607000D002E
:104298009B46036883B0042251469146BA465F465E
:1042A8009A692A40521B504242418A4200D080E01B
:1042B8002200986902409446002204420ED0DC6134
:1042C8007A1C00D07CE020209A691042FCD000269D
:1042D8002022DA614A4632439446012280209E69B0
:1042E8004000064237D06246012431005746224337
:1042F800D861700504D5082002438020C000D86129
:10430800890504D502210A43FF31FF31D961996932
:10431800890701D50021996201219869014202D1DA
:1043280098690143996159684F48014059607B6C0D
:1043380013437B6420224123FA5400220133FA54A8
:10434800402300220120FA5403B0F0BCBB46B24619
:10435800A946A046F0BD700503D562463100574610
:10436800C9E7B60502D562465746CBE7002A24D1ED
:104378007A1C95D0BB4657468A46FEF739FF0C9BF8
:10438800C01A584502D85B46002B14D13B689A697D
:104398002A40521B51424A41524500D07BE7202215
:1043A8007B6C13437B644123FA5400220133FA5493
:1043B800C6E70020C8E73B686DE762465746A6E7B0
:1043C8000C9A0026934600220092203290462A003A
:1043D8005546B2465E469346019141469A69114256
:1043E80034D1009A002A3AD1FEF702FF2B68801BCD
:1043F800874201D3002FF0D142225868AA5C9969FC
:10440800D2B294468022120211420DD08021C901F5
:10441800084209D16246202A06D05A6811435960D9
:10442800FEF7E6FE06002B6841469A691142D4D190
:10443800FEF7DEFE2B68801B1928F5D9202241469D
:1044480092461F3A00929A691142CAD0009A56467B
:104458000199AA465D46002A00D139E73AE756464F
:104468000199AA465D4635E700E800FEF0B5DE464C
:1044780057464E464546E0B50D000421036892466E
:104488009A69040010268B4683B0920664D43200E1
:10449800996900270A400E420CD0DE616A1C65D17A
:1044A80020219A691142FCD000222021D961594665
:1044B80001270A43802099694000014234D0012530
:1044C800D8612A43480504D5082002438020C0004B
:1044D800D861890504D502210A43FF31FF31D9612A
:1044E8009969890701D500219962012198690142DA
:1044F80002D198690143996159684448014059605B
:10450800636C1343636420224123E2540022013385
:10451800E254402300220120E25403B0F0BCBB4621
:10452800B246A946A046F0BD4805CDD48905D2D4E7
:10453800002FD5D1FEF75CFE5346C01A2368A84267
:1045480001D8002D05D120221000996908400A429F
:1045580004D09A6992069AD50020DEE7636C13436B
:1045680063644123E2540133E054D2E72800002277
:1045780000215546894620279246804601959A692A
:1045880017420ED14A46002A3BD1FEF731FE401BA6
:1045980080450FD34346002B0CD023689A691742F5
:1045A800F0D0019952468A4649464546002900D12D
:1045B8007BE77CE7422223685868A25C9969D2B2FB
:1045C80094468022120211420DD08021C90108426E
:1045D80009D16246202A06D05A6811435960FEF76D
:1045E80007FE050023689A691742C8D1FEF700FE46
:1045F8002368401B1928F6D9202292461F3A914673
:10460800BDE70199524645468A4650E700E800FE54
:10461800F0B557464E46DE464546E0B50368924635
:104628009A6904000E0083B0520700D595E0042271
:10463800102593462A00996900270A400D420DD09B
:10464800DD61721C00D094E020219A691142FCD0EF
:1046580000222021D961594601270A4380209969FF
:10466800400001423AD00125D8612A43480504D5C3
:10467800082002438020C000D861890504D50221A2
:104688000A43FF31FF31D9619969890701D50021B2
:10469800996201219869014202D19869014399619F
:1046A80059685C4801405960616C42200A43626461
:1046B80041212022625400212154023821549B694F
:1046C8001A4228D0FEF794FD23689B69012003B0A5
:1046D800F0BCBB46B246A946A046F0BD4805C7D4C3
:1046E8008905CCD4002FCFD1202299690A4218D04D
:1046F800996999690D4213D00421DD616164DA6119
:1047080059684448014059604123E2540133E75451
:10471800023BE754D6E7FEF76BFD23689B69D5E7B4
:104728006764FEF765FD5346C01A864217D22268B1
:1047380058465F469169130008400F4209D120216D
:10474800636C0B4363644123E154013BE054936978
:10475800BCE79269174200D16CE70020B7E72368ED
:104768001A00002EE4D09A69520700D462E70020AC
:10477800ADE73000002200215646894620279246A0
:10478800804601969A6917420ED14A46002A3BD1C3
:10479800FEF72EFD801B80450FD34346002B0CD01F
:1047A80023689A691742F0D0019952468A464946C9
:1047B8004646002900D14CE74DE742222368586855
:1047C800A25C9969D2B294468022120211420DD09D
:1047D8008021C901084209D16246202A06D05A68B8
:1047E80011435960FEF704FD060023689A691742D1
:1047F800C8D1FEF7FDFC2368801B1928F6D92022B2
:1048080092461F3A9146BDE70199524646468A4666
:1048180021E7C04600E800FE10B5041E52D041232F
:10482800C35CDAB2002B48D0412324220121E25490
:104838002368A0681A688A431A60234962680A4094
:104848001A619A6821490A409A60E268012A0BD0E5
:104858008421090201439960022A09D180225968FA
:1048680012010A435A6007E08022120202439A604A
:104878005A6817490A405A605968164A00200A437C
:104888005A60DA6811490A40DA60616922690A43A4
:10489800A16909020A43DA60216AE2690A4301212F
:1048A8001A601A680A431A60002341221F316364A0
:1048B800A15401322363A35410BD4033C254FEF700
:1048C8004DF9B1E70120F7E7FFFFFFF0FF7FFFFF9A
:1048D800FFF7FFFF00800002F0B5574645464E46F9
:1048E800DE46E0B585B01F000E9B04009A464123C2
:1048F8009846C35C0E001500202B00D08AE02033B8
:10490800C25C012A00D185E00122C254FEF770FC86
:10491800010003902000FFF70BFB002872D1212330
:104928004246A3542133313AE25460646785628D6C
:10493800B605236865626063B70DFF2A6CD8618D80
:1049480089B22185002900D059E15A68B0490A4046
:10495800B0493A430A435A60628D10255646002AE8
:1049680000D1B9E00222B9469246A34651465046C4
:104978009A691140104200D095E02A0098690024F5
:10498800024005420CD0DD61721C00D0E3E020201B
:104998009A691042FCD02022DA61042201240A43D9
:1049A800802099694000014252D001255C462A4383
:1049B800D861480504D5082002438020C000D8618A
:1049C800890504D502210A43FF31FF31D96199696C
:1049D800890701D50021996201219869014202D114
:1049E80098690143996159688B4801405960636C23
:1049F8001343636420224123E25400232232A35448
:104A0800023AA354012005B0F0BCBB46B246A94601
:104A1800A046F0BD0220F6E7FF22FF218020FE26F7
:104A28002285090440042A7801359A62628D6562FC
:104A3800013A92B262850A005D6875493A43294095
:104A48000A438021024389010A4326855A6083E785
:104A5800480501D55C46AEE7890501D55C46B1E756
:104A6800002C67D1721C00D180E7FEF7C1FB5C46C1
:104A7800039B4F46C01A2368864202D3002E00D0FB
:104A880070E7022108009A691040114200D069E7D6
:104A98002022636C134363644123E2540133E054DE
:104AA800023BE054AEE75C46626A4F461178013239
:104AB80099626262628D013A92B26285228D618D3D
:104AC800013A92B22285002901D0002A1AD0628DBB
:104AD800002A00D046E7B24651462000039AFFF765
:104AE800C5FC002800D08DE7202123684A4DD961F4
:104AF8005A682A405A604123E1540133E054023B8A
:104B0800E05480E7039B8021009320003300FFF7E7
:104B1800B5FB002800D075E7628D2368FF2A0BD902
:104B2800FF223E4922855A680A403D493A430A43D2
:104B38005A60CCE75C464AE7628D384892B25968B9
:104B48002285D2B2120401403A430A4380218904E3
:104B58000A435A60BBE7002290464A460292320056
:104B6800039C2027260089465C4693469A6917428B
:104B78000ED14246002A3CD1FEF73AFB801B834502
:104B880010D35B46002B0DD023689A691742F0D0EA
:104B9800029A4946914642465E46A346002A00D1FB
:104BA800F9E6FAE6422223685868A25C9969D2B20B
:104BB80094468022120211420DD08021C901084278
:104BC80009D16246202A06D05A6811435960FEF777
:104BD8000FFB060023689A691742C7D1FEF708FB46
:104BE8002368801B1928F6D9202291461F3A90463F
:104BF800BCE7029A49465E469146A346CDE6802028
:104C080001398EB2711CC9B2090480040BE7C04691
:104C1800009800FC0020000200E800FE009C00FC58
:104C28000000FF01F0B54646D6464F469846412358
:104C3800C0B59A46C35C82B004000E0091460A9D36
:104C4800202B00D084E02033C25C012A00D17FE011
:104C58000122C254FEF7CCFA070001002000FFF73A
:104C680067F900286DD122235246A354102220331D
:104C7800E2544B466362434660646385B605638DC0
:104C8800B20D904660632268FF2B63D84046638D5F
:104C980051689BB22385DBB21B0403433B480140A8
:104CA8000B433B490B435360638D3A0029002000B6
:104CB800002B34D0FFF7ACFC002842D123685A6A95
:104CC800636A1A70668D636A013E01336362B6B225
:104CD800238D6685013B628D9BB22385002AE3D034
:104CE800002BE1D12B000022802120000097FFF744
:104CF800C5FA002825D1638D2268FF2B35D9FF23FB
:104D080024492385536820000B4041460B43224920
:104D18000B435360638D3A002900002BCAD1FFF77B
:104D2800A5FB00280DD1202123681C4DD9615A68A4
:104D38002A405A604123E1540133E054023BE054D5
:104D480000E0012002B0E0BCBA46B146A846F0BD7A
:104D58000220F7E7FF230D49238553680B4041469E
:104D68000B430F490B4353609EE74046638D5168E0
:104D78009BB22385DBB21B040343064801400B4367
:104D8800802189040B4353608EE7C046009800FCDD
:104D980000240002009C00FC0000FF0100E800FE67
:104DA8000024FF01F0B557464E46DE464546E0B5BD
:104DB80083B01F000CAB160004CB04001B880D0049
:104DC8009B4641239946C35C9246202B1FD1002A5B
:104DD80019D05B46002B16D04022835C012B16D0DD
:104DE80001238354FEF704FA804601002000FFF7F0
:104DF8009FF800280DD0012003B0F0BCBB46B24696
:104E0800A946A046F0BD80239B006364F3E7022017
:104E1800F2E721234A46A35440222133E254534661
:104E280063625B462168606463854A6860635448CE
:104E3800FBB20240AD051B041343AD0D514A2B4391
:104E480013434B60424620000E99FFF727F90028CC
:104E580057D12368012F62D1F6B29E6243460022E1
:104E68000093802120000E9BFFF708FA002848D104
:104E7800638D2268FF2B48D8638D43489BB25168E5
:104E88002385DBB21B0401402B430B43802189049B
:104E98000B43536002E0638D002B5AD0424620003A
:104EA8000E99FFF7FBF80028A5D1636A22681978E4
:104EB800013391626362638D013B9BB26385238DED
:104EC800628D013B9BB22385002AE4D0002BE2D1FE
:104ED800434600220093802120000E9BFFF7CEF965
:104EE800002800D087E7638D2268FF2B22D9FF2393
:104EF8002549238553680B4024492B430B435360B2
:104F0800C9E740230022E25475E7FF231E492385A1
:104F180053680B401D492B430B435360BEE7320ACD
:104F28009A62200042460E99FFF7B8F80028E8D1A7
:104F3800236891E7638D14489BB251682385DBB2DF
:104F48001B0401402B430B43802189040B4353600E
:104F5800A1E7424620000E99FFF788FA002800D002
:104F680049E7202123680A4DD9615A682A405A60C6
:104F78004123E1540133E054023BE0543CE7C0468E
:104F8800009800FC00200001009C00FC0000FF01CC
:104F980000E800FEF0B557464E46DE464546E0B509
:104FA80083B01F000CAB160004CB04001B880D0057
:104FB8009B4641239946C35C9246202B1FD1002A69
:104FC80019D05B46002B16D04022835C012B16D0EB
:104FD80001238354FEF70CF9804601002000FEF7F8
:104FE800A7FF00280DD0012003B0F0BCBB46B24695
:104FF800A946A046F0BD80239B006364F3E7022026
:10500800F2E722234A46A35440222033E25453466F
:1050180063625B462168606463854A6860635648DA
:10502800FBB202401B0413438022AD05AD0D920173
:105038002B4313434B60424620000E99FFF72EF88E
:1050480000285AD12368012F65D1F6B29E624346E3
:1050580000220093402120000E9BFFF70FF9002843
:105068004BD1638D2268FF2B4BD8638D42489BB28E
:1050780051682385DBB21B0401402B430B433F4996
:105088000B43536002E0638D002B5ED04346002241
:105098000093042120000E9BFFF7F0F80028A2D10E
:1050A80023685A6A636A1A70628D636A013A013327
:1050B80092B26362238D6285013B628D9BB2238528
:1050C800002AE0D0002BDED1434600220093802145
:1050D80020000E9BFFF7D2F8002800D083E7638DED
:1050E8002268FF2B22D9FF232549238553680B40CB
:1050F80024492B430B435360C5E740230022E25465
:1051080071E7FF231C49238553680B401E492B4335
:105118000B435360BAE7320A9A62200042460E995E
:10512800FEF7BCFF0028E8D123688EE7638D14489A
:105138009BB251682385DBB21B0401402B430B4310
:10514800802189040B4353609DE7424620000E9955
:10515800FFF78CF9002800D045E7202123680B4D84
:10516800D9615A682A405A604123E1540133E05416
:10517800023BE05438E7C046009800FC00240002D7
:10518800009C00FC0000FF010024FF0100E800FE75
:10519800F0B54546DE4657464E46E0B51D000023AD
:1051A8009046412287B00593835C0400202B57D199
:1051B800036880209E6900023700074006424FD1ED
:1051C8004020265C012E4BD0012626541C38A054C2
:1051D80067648F05BA0D110003923E4A1143894650
:1051E800E1684A46012902D13B4A03990A435A60B9
:1051F800FDF7FEFF202322680600916990690B40A5
:10520800102101400B4309D16B1C31D120271020FC
:1052180091699369394003401943F9D09369102281
:10522800009692461A4244D02B00002220212000EA
:10523800FFF724F8002811D1524620212368DA61AB
:10524800D961059A01320592059A4245C8D341238E
:10525800E154636C0B4363644023E054012000E095
:10526800022007B0F0BCBB46B246A946A046F0BD36
:10527800002D1BD0202310279B4607E058462268A4
:1052880093699169034039400B43C7D1FDF7B0FFDB
:10529800801B8542F2D220224123E254636C012014
:1052A8001343636400224023E254DAE7FDF7A0FFCA
:1052B800F1E72B00002220212000FEF7DFFF002865
:1052C800CCD120232268D3614122A3542033E05457
:1052D800C7E7C0460028000200200002F0B54124BC
:1052E800035D8C46DDB2202B1AD14026835D012B4D
:1052F80016D024230127035503680A491A68BA43BC
:105308001A601A680A401A606246196811431960DF
:105318001A683A431A600023055583550020F0BDEA
:105328000220FCE7FFEFFFFFF0B5CE4647464124D9
:1053380080B5035DDDB2202B1FD14026835D012B94
:105348001BD02423012703550268B94613680902B4
:10535800BB431360136898464746094B1F403943BF
:105368001160494613680B431360002305558355A4
:105378000020C0BCB946B046F0BD0220F9E7C046DF
:10538800FFF0FFFF70B5041E23D00368144A1A60AB
:10539800144A1A6042685A6082689A60FDF728FFCA
:1053A80023680600DA6852070CD00725FDF720FFAE
:1053B8002368801B312802D9DA6815420BD1DA68D4
:1053C8001542F3D11969E268914206D01A610020AA
:1053D80070BD0120FCE70320FAE7034A1A60F6E7EC
:1053E800CCCC000055550000AAAA00000368024A68
:1053F80000201A607047C046AAAA000070B5134C76
:10540800134A2368002513400343236080239B002D
:10541800984201D0280070BD0E4B0F491B685800F8
:10542800C0184000FAF768FE80226369D200013094
:10543800134202D1EEE7002805D063690138134210
:10544800F9D10025E6E70325E4E7C04600700040EF
:10545800FFF9FFFF0000002040420F00F0B5CE46E4
:10546800474680B5040083B0002827D00368DA07D0
:1054780011D53822C0498868C9680240102A00D16D
:10548800CCE0082A00D0CDE0BB4A1268920302D5CE
:105498006268002A12D09A0732D53823B64A916832
:1054A8000B40D168102B00D10BE1002B00D00DE18F
:1054B80013685B0508D5E368002B05D1012003B00C
:1054C800C0BCB946B046F0BD51686369AB481B0221
:1054D80001400B435360A84AA94913680B4021694E
:1054E8000B4313601368A74A9B045B0FDA40A64975
:1054F8000A60A64B1868FDF735FE0028DED1236840
:105508001A076DD45B0745D538239B4A91680B4031
:10551800202B00D1CCE080230020D16B5B05814695
:10552800194208D1D16B1943D163D26B134001934F
:10553800019B012399468027954E7F0033683B42A3
:1055480000D1FFE0A368012B00D1E5E0052B00D1D5
:10555800C8E10121884EF26D8A43F265F26D03318C
:105568008A43F265002B00D0DAE0FDF741FE022302
:1055780007009846874D05E0FDF73AFEC01BA84294
:1055880000D9EEE04246F36D1A42F5D14B46012BA5
:1055980000D163E1E369002B20D03822764DA96859
:1055A8000A40102A00D11DE1022B00D15CE12B68D2
:1055B800794A802613402B60FDF71AFEB6040400D2
:1055C80005E0FDF715FE001B022800D9C9E02B688D
:1055D8003342F6D1EB68714A1340EB6000206EE766
:1055E8003822654DA9680A40182A43D0A369002BC0
:1055F80000D1B8E001222B6E022713432B66FDF77A
:10560800F7FD060005E0FDF7F3FD801B022800D931
:10561800A7E02B6E1F42F6D0236873E7C9438907BA
:1056280000D131E780226368520293422BD0A02137
:10563800C9028B4200D1FCE04F4D59492A680A4003
:105648002A602A6857490A402A60002B1FD1FDF7B3
:10565800CFFD80270600BF0204E0FDF7C9FD801BCF
:1056680064287ED82B683B42F7D123689A0700D478
:1056780046E712E72A6E920700D443E7A269002A98
:1056880000D03FE71AE73C4A11680B431360FDF767
:10569800AFFD80260500384FB60204E0FDF7A8FDEF
:1056A800401B64285DD83B683342F7D02368DDE7A8
:1056B800D36D9B0700D46DE7A368002B00D069E782
:1056C800FCE60D3B0B40022B00D1BCE0E3682A4D01
:1056D800002B73D02B682A4A802713402269FF00C9
:1056E80013432B6080232A685B0013432B60FDF76C
:1056F8007FFD060004E0FDF77BFD801B022830D803
:105708002B683B42F7D06A6863691C491B020A4050
:1057180013436B602368F3E61749CA6D1343CB65DF
:10572800FDF766FD144B060098460227194D04E064
:10573800FDF75EFD801BA84213D84346DB6D1F4270
:10574800F6D023E733683B433360FDF751FD05008E
:1057580033683B4200D0F5E6FDF74AFD401B0228BE
:10576800F6D90320ABE601222B6E022793432B6662
:10577800FDF73EFD06001CE000100240FF80FFFF21
:10578800FFC7FFFF0024F4000000002008000020ED
:105798000070004088130000FFFFFFFEFCFFFEEFD3
:1057A800FFFFFEFFFFFFFBFFFDF722FD801B022826
:1057B800D7D82B6E1F42F7D12368A3E62B68504A2F
:1057C800802713402B60FDF713FDFF00060004E05F
:1057D800FDF70EFD801B0228C3D82B683B42F7D18A
:1057E80023688DE6012B00D168E60322E868216A68
:1057F80002408A4200D061E67022616A02408A4211
:1058080000D05BE6FE21A26AC90101401202914262
:1058180000D053E6F822E16A920302408A4200D09F
:105828004CE6236B400F4007C01A431E9841C0B294
:1058380045E68021334BC90218680143196019688D
:105848000A431A6023E713685B0555D451686369F6
:105858002D481B0201400B4353604AE6294A2B4955
:10586800D36B0B40D36395E62B68294A80271340F6
:105878002B60FDF7BDFCBF04060005E0FDF7B8FC92
:10588800801B022800D96CE72B683B42F6D1616A7D
:10589800236AEA680B431F491A4E0A401343E26A17
:1058A8001343226B1343A26A12021343EB60802353
:1058B8002A685B0413432B608023EA685B05134363
:1058C800EB60FDF795FC80250400AD0405E0FDF7CD
:1058D8008FFC001B022800D943E733682B42F6D01F
:1058E8000020ECE50421074BDA6D0A43DA65DA6D2E
:1058F80003390A43DA6513E7E368002BA6D1DDE52F
:10590800FFFEFFFF00100240FF80FFFFFFFFFFEFD9
:10591800FFFFFFFE8C80C11F3823224A10B5916813
:105928000B4205D1136820489B045B0FD84010BD7B
:1059380091681940082914D091681940102912D08B
:1059480091681940202924D0906818401838431EBF
:105958009841164B40421840FA23DB019C466044AC
:10596800E5E71348E3E7D368D168DB43D468490621
:10597800490F64040131640E9B070DD00A48FAF7F9
:10598800BBFB6043074BD968490F0131FAF7B4FBF9
:10599800CDE780200002CAE70548FAF7ADFB60436F
:1059A800F0E7C046001002400024F4000083FFFF27
:1059B80000127A00F8B5CE46474605000C0080B5BF
:1059C800002826D00722574E336813408B425ED3F7
:1059D8002B689A070ED55A0705D5E0225249D201FD
:1059E800886802438A60504950488A680240A8681B
:1059F80002438A60DB072BD56B684B4A012B00D129
:105A08007CE0022B07D0002B00D07DE01268520505
:105A180004D4012037E012689201FAD50721424EDA
:105A2800B2688A431343B360FDF7E2FB3823984614
:105A38003F4B0700994604E0FDF7DAFBC01B4845D9
:105A48003BD84346B2681A406B68DB009A42F3D1F0
:105A58000722344E33681340A34238D82B685B07BB
:105A68002DD4FFF759FF304B324A9B6832491B054A
:105A78001B0F9B009B581F221340D8402F4B0860D8
:105A88001868FDF76FFBC0BCB946B046F8BD33686F
:105A980093430B433360FDF7ABFB07239846244B36
:105AA80007009946424633681340A34200D18FE766
:105AB800FDF79EFBC01B4845F4D90320E3E71A4ACB
:105AC8001F4993680B40E9680B439360C9E7336843
:105AD800934323433360FDF78BFB07239846144B0E
:105AE80007009946424633681340A342B6D0FDF7F3
:105AF8007FFBC01B4845F5D90320C4E71268920311
:105B080000D58BE70120BEE7032B05D0D26D9207A5
:105B180000D583E70120B6E7126E920700D57DE72E
:105B28000120B0E70020024000100240FFF0FFFF14
:105B38008813000060820008000000200800002090
:105B4800FF8FFFFF064B07499B68074A5B045B0F03
:105B58009B005B581F2110680B40D8407047C04617
:105B6800001002404082000800000020F0B5D64630
:105B78004F464646C0B50368040082B000209A0329
:105B880051D58022564B5205D96B8246114200D11D
:105B980084E08027534D7F002B683B432B60FDF743
:105BA80027FB060005E0FDF723FB801B022800D930
:105BB8007EE02B683B42F6D0494DC023EA6D9B003E
:105BC8001000A16918401A4222D0884220D08020B3
:105BD800EB6DEE6D40023043E865E86D424A434E96
:105BE8001A403040E865EA65DB0711D5FDF700FB90
:105BF800022398463E4B0600994604E0FDF7F8FA62
:105C0800801B484554D84246EB6D1A42F6D0A1692C
:105C1800334A3548D36D03400B43D36552460020C1
:105C28002368012A49D0DA0706D503252C494A6D8D
:105C3800AA4365682A434A659A0706D50C25284968
:105C48004A6DAA43A5682A434A659A0606D5244997
:105C5800284D4A6D2A40E5682A434A655A040AD500
:105C68001F4965694A6D920092082A434A65802255
:105C7800D205954227D01B050AD5194A2169536DCB
:105C88001D4C23400B4353658023DB01994220D0F0
:105C980002B0E0BCBA46B146A846F0BDD96B114384
:105CA800D963DB6B13400193019B01239A4670E78C
:105CB800524603202368012AB5D109490F4DCA6B02
:105CC8002A40CA63AFE78022CD6852022A43CA60DD
:105CD800D1E78023D1685B020B43D360D8E7C04685
:105CE8000010024000700040FFFCFFFFFFFFFEFFB6
:105CF80088130000FFCFFFFFFF3FFFFFFFFFFFEF0D
:105D080070B5041E00D171E03D23C35CDAB2002BEC
:105D180020D03D230222E2542368354E1A68616878
:105D2800E068A569B3421AD0324EB3424AD0324E27
:105D3800B3424BD0314EB3424DD0314EB34212D064
:105D4800304EB3420FD08026B2432A431A60D8623D
:105D5800996214E03C33C254FDF774F8D9E7702611
:105D6800B243A6683243284E324026693243802621
:105D7800B2432A431A60D862996262691A6301229F
:105D88005A6119690A4202D01969914319610123BC
:105D980048220020A3540A3AA3540132A3540132E2
:105DA800A3540132A3540132A3540132A354013243
:105DB800A3540132A3540132A3540132A3540A3A22
:105DC800A35470BD7026B243A66832430E4E3240CB
:105DD80026693243B7E70C4E3240266932438026A3
:105DE800B24315431D60D8629962C6E70120E8E70F
:105DF800002C014000040040002000400040014009
:105E08000044014000480140FFFCFFFF13008822C6
:105E1800F0B5C6468258040000B5202A2CD10029C6
:105E280028D0002B26D0802280685201904238D09A
:105E380054222165A3520232A35232329046902650
:105E480040460027673AA7512250E06F2268002891
:105E580017D0174D8763C562164D28320563164D56
:105E68004563FDF727FE00280AD010234246A351B8
:105E78001033A350012000E0022080BCB846F0BDDA
:105E8800226840231362EFF310813F3B83F31088AD
:105E98008020226893680343936081F31088002070
:105EA800EBE72269002AC3D1CA07C1D50120E4E77C
:105EB800F96000084D61000865610008F8B50D003B
:105EC8008C214158040020295FD1002D0BD0002AD5
:105ED80009D0802381685B01994206D10369002BB0
:105EE80003D1EB0701D501204EE00023E3662368C8
:105EF8005B681B020CD5EFF31080012383F3108835
:105F080080232168DB040E6833430B6080F310881C
:105F18005C23A5652221E252902700238C26E351B9
:105F2800A1515E316058002814D01F498363C162B3
:105F38001E49130001631E492A0041632168243168
:105F4800FDF7B8FD002805D01023E35110330120D8
:105F5800A35119E02369002B19D1EFF31080012315
:105F680083F3108821688A681A438A6080F310884E
:105F7800EFF3108183F3108840202268936803436D
:105F8800936081F310880020F8BD0220FCE7EFF34E
:105F98001081012383F310882268FF3310680343BC
:105FA800136081F31088D8E749660008296600085D
:105FB80065610008882370B504008022C058043346
:105FC800E558236899680A4201D0212846D09A6882
:105FD8004023134201D1002070BD222DFBD1EFF3E5
:105FE8001080012282F3108821688A689A438A60A7
:105FF80080F3108880256059002803D0FDF7C2FD82
:1060080000285ED1EFF31080012282F31088216806
:10601800344D0B682B400B6080F31088EFF3108130
:1060280082F310882268304893680340936081F3B4
:106038001088E36E012B0AD1EFF3108183F31088E7
:106048001020226813688343136081F310888C231F
:106058002022E2500023E3666367BCE7EFF3108079
:10606800012383F3108821688B6893438B6080F346
:106078001088E06F002803D0FDF784FD00282AD19E
:10608800EFF31080012282F31088C02621680B6884
:10609800B3430B6080F31088EFF3108182F310880C
:1060A8002268124893680340936081F3108888231C
:1060B8002022E25023689A684023134200D18AE7DD
:1060C8008BE76059FDF732FE20289BD190231022E0
:1060D8000320E25080E7E06FFDF728FE2028CFD1AB
:1060E800F4E7C046DFFEFFFFFEFFFFEFFFFF7FFF85
:1060F8002022030011001B6810B51B68806A194034
:106108001A4219D15623C152EFF3108C1F3A82F369
:106118001088802401688B68A3438B608CF31088F7
:10612800EFF3108182F3108802684020136803435C
:10613800136081F3108810BD01F02EFAFBE7C0460A
:106148007047C04610B5806AFFF7FAFF10BDC04619
:106158007047C0467047C0467047C046F8B58821AA
:106168008C23806A4558C45803689A68120601D57A
:10617800212D0CD09B685B0601D5222C25D09022BE
:10618800102183580B438350FFF7E6FFF8BD5623D1
:106198000022C252EFF31086013282F31088C02722
:1061A80005682B68BB432B6086F31088EFF31085D6
:1061B80082F3108802681C4E93683340936085F31D
:1061C8001088202343500368D4E75E230022C2527C
:1061D800EFF31084013282F310880168134D0B68C5
:1061E8002B400B6084F31088EFF3108182F3108842
:1061F80002680F4C93682340936081F31088C36E44
:10620800012B0AD1EFF3108183F310881024026860
:106218001368A343136081F310888C232022C25093
:106228000023C3664367AAE7FFFF7FFFDFFEFFFF88
:10623800FEFFFFEF00235E2210B5806A8352083A02
:106248008352FFF789FF10BD7047C046F8B5454631
:10625800DE4657464E460268E0B5D369AE4D0400A7
:10626800116890682B4238D120251D4206D080261F
:1062780076050D400640354300D015E1E56E012D49
:1062880000D1D8E080256D032B421FD180221A420D
:1062980006D080252D040A402840024300D00AE198
:1062A80040221A4202D00A4200D014E11A0202D552
:1062B8004A0000D523E1DB0102D5002900DA22E1FA
:1062C800F0BCBB46B246A946A046F8BD4602DDD59D
:1062D8002000156200F0B4FCF2E7904E904D0640A5
:1062E8000D403543CAD001251D4208D0CF0506D53B
:1062F8009027BC461562E7593D436746E55104259A
:106308002F001F40BC460227A9461F4200D1C3E008
:10631800C50716D5902517626759A8464D463D43CF
:106328004746E5516546002D0BD0042515628C358E
:10633800A9466559A846022547462F433D004F46C2
:10634800E55108271F4208D020250D40354304D0C9
:1063580090261762A5593D43A55180252D012B4252
:1063680007D04E0105D5902620271562A5593D4333
:10637800A55190256559002DA2D020251D4206D093
:1063880080235B050D4003401D4300D097E0902615
:106398004025A15993681D4028230B401D4300D177
:1063A800B5E0EFF31080012282F3108821685D4D7B
:1063B8000B682B400B6080F31088EFF3108182F399
:1063C80010882268584893680340936081F31088C6
:1063D800E36E012B0AD1EFF3108183F310881020AC
:1063E800226813688343136081F310888C2320226A
:1063F800E2500023E3666367236820329B681A42F1
:1064080065D0EFF31080012383F3108821688B682F
:1064180093438B6080F3108880256059002856D0FC
:10642800424B8363FDF7EAFB002800D148E7605937
:10643800836B984744E710261E4200D122E70E429C
:1064480000D11FE7402318001662926810401342DB
:106458006ED080229446A2581068426892B2002AF0
:1064680000D12DE75C218B46615A914200D827E77D
:106478005E27E2532022170000680740B846024210
:1064880000D192E0022323675C33E35A2000C91A43
:1064980089B2FFF7D9FE13E76546002D00D150E712
:1064A800C50700D44DE740E7636F002B00D107E72D
:1064B8002000984704E7A36F002BF9D100E7636F2A
:1064C800002B00D163E72000984722685FE720008F
:1064D800FFF742FEF4E6EFF31080012383F3108800
:1064E80021680B6893430B6080F310888823203A57
:1064F800E25000232000A36701F04EF8E0E62000F8
:1065080000F0A2FBDCE6200000F09CFBD8E62000AF
:10651800FFF722FEA551D3E60F0800000100001086
:1065280020010004DFFEFFFFFEFFFFEF3D620008D1
:106538005C235E22E15AA35AA25A9BB2002A00D1D8
:10654800BEE6C91A89B2002900D1B9E6EFF310896D
:1065580085F3108822681368984647462D4B1F40DC
:10656800176089F31088EFF3108985F31088226883
:10657800936898464746284B1F40976089F31088D0
:106588008C232022E250E0666067EFF3108085F3E9
:10659800108822681368B343136080F310880223BD
:1065A80020002367FFF750FE8AE6EFF3108985F392
:1065B80010882068194F01683940016089F31088F4
:1065C800EFF3108985F3108820688168A9438160FA
:1065D80089F31088EFF3108985F3108820688168A3
:1065E8009943816089F310884C33E2504346E3664F
:1065F800EFF3108185F3108822681368B3431360A2
:1066080081F310886346E058FDF7BCFA5B46E15A0F
:1066180038E7C046DFFEFFFFFEFFFFEFFFFEFFFF8C
:106628000123806A10B50367C36E012B02D0FFF700
:1066380091FD10BD5B33C15A4908FFF705FEF8E725
:1066480003001B6870B51A6820231900806A11407E
:10665800134227D15E228152EFF310855D3A82F30F
:10666800108804681C4E21683140216085F3108829
:10667800EFF3108582F310880468A1689143A16044
:1066880085F31088EFF3108482F3108840250168A1
:106698008A68AA438A6084F310888C228350C36E68
:1066A800012B0CD000230367C36E012B02D0FFF728
:1066B8004FFD70BD5B33C15AFFF7C6FDF9E7EFF335
:1066C800108183F31088102402681368A3431360B1
:1066D80081F31088E6E7C046FFFEFFFF836A30B506
:1066E8001A0706D50168284C4A682240846B224361
:1066F8004A60DA0706D50168244C4A682240C46A11
:1067080022434A609A0706D50168214C4A6822400C
:10671800046B22434A605A0706D501681D4C4A6833
:106728002240446B22434A60DA0606D501681A4CB7
:106738008A682240C46B22438A609A0606D501689B
:10674800164C8A682240046C22438A605A060AD58D
:106758000168134D4A68446C2A4022434A608022EB
:106768005203944209D01B0606D502680D495368A6
:106778000B40C16C0B43536030BD4A680A4C224041
:10678800846C22434A60EEE7FF7FFFFFFFFFFDFFB7
:10679800FFFFFEFFFFFFFBFFFFEFFFFFFFDFFFFF36
:1067A800FFFFEFFFFFFFF7FFFFFF9FFFF0B590230D
:1067B8000022C646040000B5C250FCF719FD236844
:1067C80005001A68120711D41A6852073ED420230C
:1067D8008822A3500432A35000230020E3662367D5
:1067E80084230022E25480BCB846F0BDDA699202E4
:1067F800EAD48026082304279846B60410E02368C4
:106808001A68174209D04146DA69114259D18022E3
:10681800D9691201114200D085E0DA699202D3D415
:10682800FCF7E6FC401BB042E9D3EFF310810123EB
:1068380083F310888020226813688343136081F3F0
:106848001088882320220320E250C9E7DB695B0215
:10685800BDD48026082304279846B60411E023688F
:106868001A6817420AD04146DA69114200D08BE013
:106878008022D9691201114200D0B7E0DB695B02BE
:10688800A5D4FCF7B5FC401BB042E8D3EFF3108069
:10689800012282F3108821686D4D0B682B400B6034
:1068A80080F31088EFF3108082F3108821688B68DA
:1068B80093438B6080F310888C231F320320E250AF
:1068C8008EE71962EFF31080012282F310882168A5
:1068D8005F4D0B682B400B6080F31088EFF310813D
:1068E80082F3108822685B4893680340936081F3C1
:1068F8001088E36E012B0AD1EFF3108183F310881F
:106908001020226813688343136081F310888C2356
:1069180020220821E25000237032E3666367A15009
:106928000C3AA35481E71A62EFF31080012282F334
:1069380010882168464D0B682B400B6080F3108847
:10694800EFF3108182F3108822684248936803406D
:10695800936081F31088E36E012B0AD1EFF3108165
:1069680083F310881020226813688343136081F32F
:10697800108820228C239021E2500023E36663676D
:1069880062506432A35450E71962EFF31080012279
:1069980082F3108821682E4D0B682B400B6080F322
:1069A8001088EFF3108182F31088226829489368D1
:1069B8000340936081F31088E36E012B0AD1EFF353
:1069C800108183F3108810202268136883431360B2
:1069D80081F310888C2320220821E2500023703292
:1069E800E3666367A1500C3AA3544FE71A62EFF3CA
:1069F8001080012282F310882168154D0B682B4006
:106A08000B6080F31088EFF3108182F310882268FE
:106A1800104893680340936081F31088E36E012B5C
:106A28000AD1EFF3108183F31088102022681368CD
:106A38008343136081F3108820228C239021E25035
:106A48000023E366636762506432A3541EE7C046BE
:106A5800DFFEFFFFFEFFFFEF70B5041E41D0882365
:106A6800C358002B00D17DE0882324222568E250FA
:106A78002B68233A93432B60A36A002B00D06DE068
:106A88002169A3682A680B436169E0690B435E4981
:106A980003430A4013432B606B685C4A216A134026
:106AA800E26813436B60A369AA680B4358490A401C
:106AB8000F211343AB60EB6A626A8B431343EB62AB
:106AC800544B9D420FD0544B9D4250D0534B9D4246
:106AD80014D0534B9D4211D0524BA36600236367D9
:106AE800A367012070BD504B596D03230B40022B47
:106AF80000D17DE0032B75D0012B43D080231B02EE
:106B080098424DD0FFF71EF8002843D0626A474BE1
:106B18005200D15AF9F7F0FA65686B08C0182900D5
:106B2800F9F7EAFA0200424B103A9A42D4D823689D
:106B3800D8603C4AA26600226267A2675A683D494B
:106B480020000A402A215A609A688A439A601A6883
:106B580029390A431A60FFF729FEC3E72000FFF727
:106B6800BDFD8DE784228354FCF7E8F97CE72E4BC2
:106B7800596D0C230B40082B3AD030D8002BBDD0D0
:106B8800042BA9D180231B02984237D0FEF7C4FEFC
:106B98000028BBD1234B6067A366A0672368CDE7B5
:106BA800FEF7D0FF0028F5D0626A204B5200D15A78
:106BB800F9F7A2FA656840006B08C0182900F9F7D0
:106BC8009BFA02001A4B103A9A4200D984E71A4AF3
:106BD800236802400007400F0243DA60A9E70C2B44
:106BE80000D079E780231B029842DED018008EE798
:106BF80080231B02984204D0104888E7FEF78CFED9
:106C0800D0E70E48D1E7C046F369FFCFFFCFFFFFBB
:106C1800FFF4FF11003801400044004000480040E4
:106C2800004C00400100010000100240A082000852
:106C3800EFFF0000FFB7FFFFF0FF00000024F400A3
:106C48007047C0467047C0467047C04670B5842438
:106C5800035D012B12D088252423012643510368A4
:106C68001A681968B143196005490A40002141664C
:106C78001A60202343510155002070BD0220FCE713
:106C8800FFFFFFDFF0B5D6464F4646468423C0B522
:106C9800C35C04000A00012B3DD088232421056829
:106CA800C1502E682B6823398B432B60AB68DB00FF
:106CB800D908436E1143A960002B29D0AB68174A45
:106CC80098469246AB685B0FD05C154AC000D15C11
:106CD8009146F9F79BFA434652461B015B0F87B270
:106CE800D05C4A46C000D15CF9F790FA80B26823BC
:106CF8002022E0520233E7521E332E60E250002277
:106D08000020043BE254E0BCBA46B146A846F0BDB8
:106D180001200127EBE70220F5E7C046C082000802
:106D2800B8820008F0B5D6464F4646468423C0B51B
:106D3800C35C04000A00012B3DD088232421056888
:106D4800C1502E682B6823398B432B60A9681B4BD5
:106D58001940436E1143A960002B29D0AB68184A2B
:106D680098469246AB685B0FD05C164AC000D15C6F
:106D78009146F9F74BFA434652461B015B0F87B21F
:106D8800D05C4A46C000D15CF9F740FA80B268236B
:106D98002022E0520233E7521E332E60E2500022D6
:106DA8000020043BE254E0BCBA46B146A846F0BD18
:106DB80001200127EBE70220F5E7C046FFFFFFF1BE
:106DC800C0820008B8820008002370B54371FF3301
:106DD8000D00FF3351001940373B0270FF3B0A2278
:106DE80004000548FEF7D4F9FA222B1C52009542FC
:106DF80000D2131CE38070BD4C01002070B543889D
:106E080004000A339BB284B043800A2B06D9427926
:106E1800002A0BD0962B01D9012A23D0E2889A4266
:106E280002D200236371638004B070BD01234371F3
:106E380032330578038101000D2003AE7933083120
:106E480002326844337001F0B3F801235B420093C7
:106E58003200043369005548FDF73EFD431E984152
:106E68002071E1E7022305000126017843714900FA
:106E780008331C35314300932A004C4889B2033B40
:106E8800FDF7D0FE00285CD12100FF2331222071BC
:106E9800223128E05B00D8B25BB2002B2EDB430026
:106EA800D8B25BB2002B2FDB4000C3B240B200283F
:106EB80030DB5B00D8B25BB2002B31DB4000C3B2E1
:106EC80040B2002832DB5B00D8B25BB2002B33DB68
:106ED8004000C3B240B25B00002800DA53400135DD
:106EE800DBB2A94232D02878434058B20028D1DA20
:106EF8005800504043B2C0B2002BD0DA4000504096
:106F080043B2C0B2002BCFDA4300534058B2DBB2D1
:106F18000028CEDA5800504043B2C0B2002BCDDA78
:106F28004300534058B2DBB20028CCDA5800504036
:106F380043B2C0B2002BCBDA4300534058B2DBB2A5
:106F4800C9E700232671236363636DE72222A25CED
:106F58009A4200D068E76722237F9343182B00D01A
:106F680062E7A07F637F0002184340BAE57F80B2E2
:106F7800000228180009F9F775FD0D49F9F770FAAC
:106F88000F2220232063E35C2A4012029B1821224F
:106F9800A05C1B02C018F9F765FD0649F9F760FA0D
:106FA8000549F9F79BFB60633EE7C0464C010020AA
:106FB8000000C8380000483900004842F0B557467C
:106FC8004E46DE464546E0B587B00600171E0591D9
:106FD80030D0194B00259B460F239A46102399461B
:106FE8000A23984608E06519A619ADB20530B6B26D
:106FF800FCF704F9AF421DD954464B4634401C1BDC
:10700800A4B27B1BA34200DA9CB243460293059BC1
:1070180032005B190093A021012358460194FDF723
:10702800C1FE0028DFD007B0F0BCBB46B246A94677
:10703800A046F0BD0020F6E74C010020012310B562
:10704800064C84B05B420293019200910200A02199
:1070580020000233FDF79EFF04B010BD4C01002054
:107068000A2310B50322A0210348FEF791F8431E16
:107078009841C0B210BDC0464C010020F0B557463B
:107088004E464546DE46E0B50B4F8DB00222BB5E4C
:10709800380098460422BB5EBA469C460823FE5E2A
:1070A8000623FD5E054B624699464146B9443400C5
:1070B8002F000C300CE0C046200500205A020000CA
:1070C8001DB2C3889E4216DA1EB20A30484518D04F
:1070D8000388994200DB32E219B243889A4200DB06
:1070E80027E21AB283889D42EADB9F42E9DD1FB29C
:1070F800C3889E42E8DB9C42E7DD0A301CB2484563
:10710800E6D1230044468846614694463A005746ED
:10711800DB48385ADB4F019038880697404400B264
:107128003880D94F0290079738003F8867443FB2AC
:10713800BB46070058463880D44F00973F887D19D2
:10714800009F28B23880D24F81463D880897AD19F4
:107158002DB23D80CF4F3E880997361934B23C8016
:107168000494CD4C27880A947F18CC493FB20E88E6
:107178002780B61836B20E80C94A884614889246C7
:10718800E41824B21480C74A1388012B00D8DEE122
:107198000023032113800298F9F738F8032102B27B
:1071A80058460292F9F732F8032102B2484693464C
:1071B800F9F72CF8032102B204980B92F9F726F894
:1071C800032102B238009146F9F720F8032102B2F0
:1071D80030000492F9F71AF80023B34F0321BB805B
:1071E80006B2FB802800F9F711F8032105B2200048
:1071F800F9F70CF800B22D1AAC48AD496843F9F715
:1072080005F800B23881388900B2FBF7D7FAA94AE5
:10721800A94BFAF711FCA94AA94BFAF7D5FE0022A7
:10722800A84BFAF709FCFBF78DFA00B23881A64A99
:107238003B890020115E1BB25B1AD8171B1843400C
:107248001D2B00DC81E13B8913803B89783B1BB215
:107258003B813B891BB2002B01DA00233B814A4664
:107268003B8992481BB27B81029B91499B1A5843E8
:10727800F8F7CCFF00B2B881BB8994481BB25843D9
:107288009349F8F7C3FF00B2B881924ABB8900203E
:10729800115E1BB25B1AD8171B1843401D2B00DD6B
:1072A8005FE1B9815B46049A80489B1A584380493C
:1072B800F8F7ACFF00B2F881FB8984481BB2584349
:1072C8008349F8F7A3FF00B2F881834AFB890020BD
:1072D800115E1BB25B1AD8171B1843401D2B00DD2B
:1072E8003CE1F9810B9B71489E1B71497043F8F78B
:1072F8008DFF00B238823B8A74481BB258437449E8
:10730800F8F784FF00B23882744A3B8A0020115E85
:107318001BB25B1AD8171B1843401D2B00DD1AE15E
:107328003982B88900B2FBF749FA02900391F889CB
:1073380000B2FBF743FA0400388A0D0000B2FBF7ED
:107348003DFA22002B000490059120002900FAF74D
:1073580073FB04000D000298039902000B00FAF772
:107368006BFB02000B0020002900F9F7BDFB0400AD
:107378000D000498059902000B00FAF75DFB020066
:107388000B0020002900F9F7AFFB00F01AFEFBF70D
:10739800D9F90023069A524C1380079A00B2138039
:1073A800009A78821380089A26001380099A200090
:1073B80013800A9A01211380424613805246138093
:1073C800484B494D2360E023DB00A3800E23A371C3
:1073D800BB8915361BB21B12E371BB892372FB896B
:1073E8001BB21B126372FB89A3723B8A1BB21B126E
:1073F800E3723B8A23737B8A1BB21B1263737B8AFB
:10740800A3737B891BB21B12E3737B892374BB8A2A
:107418001BB21B126374BB8AA374FB8A1BB21B12B8
:10742800E374FB8A2375314B027853405A0819429A
:1074380001D06A4092B25308114201D06B409BB20E
:107448005A08194201D06A4092B25308114201D039
:107458006B409BB25A08194201D06A4092B2530855
:10746800114201D06B409BB25A08194201D06A40C0
:1074780092B2530811423BD06B409BB238E0C046F1
:107488004E020000E8040020E6040020E404002086
:10749800E2040020E0040020DE040020DC040020D8
:1074A800DA040020D804002004050020E40C0000C1
:1074B800FF0F0000C139234A7B83BF3FAB3E575BB8
:1074C800B1BFD43F00005940D604002050C300008B
:1074D80030390000D4040020D2040020D004002059
:1074E8007C0900200110100001A0FFFFFFFF000031
:1074F8000130864298D1224D63751B0AA3752A680C
:10750800204B9A4230D0172221002800FEF77EFC3B
:107518006B461D4804229B5E1C495843F8F776FECB
:1075280000B238830DB0F0BCBB46B246A946A046AF
:10753800F0BD9C4500DCD5E51BB29C46D2E59845DC
:1075480000DCCAE51BB29846C7E539817DE6013300
:107558000F4F1380DCE73B8A1380E2E6FB89138038
:10756800C0E6BB8913809DE6012202210948FCF789
:10757800D1FC172221002800FEF748FCC8E7C046C6
:107588000004002000380140E40C0000FF0F000058
:107598000405002000040050054B026810B59A420B
:1075A80000D010BD002202210248FCF7B3FCF8E726
:1075B8000038014000040050F0B55746DE464E46FC
:1075C8004546E0B5A14D83B06C88290064BAA3B2E2
:1075D8000193AB889E485EBA9B46B3B29A46012394
:1075E8009C4EAF1D0A7872405408134201D04440A3
:1075F800A4B26608234201D04640B6B272083342AC
:1076080001D0424092B25608134201D04640B6B269
:107618007208334201D0424092B25608134201D058
:107628004640B6B27208334201D0424092B2560880
:10763800134201D04640B6B201318F42D2D1864BB7
:10764800162218008549994600F0B2FC019B534464
:107658000C2B03DCAA79F3B29A4206D003B0F0BC33
:10766800BB46B246A946A046F0BDEA79330A9A421B
:10767800F4D17B4B984642462B88138053465B00D7
:1076880093705B46002B00D1D9E04B4644460198E5
:10769800023B4200D25E111222715246E170012A69
:1076A8006ED9421C5200D25E1112A2718022617101
:1076B8009200934564D0821C5200D25E111222724D
:1076C800C022E171920093455AD0C21C5200D25E8A
:1076D8001112A27280226172D200934550D0021D0D
:1076E8005200D35E1A122373A023E272DB009B457B
:1076F80046D05C4B421D5200D25E1112A273C022CA
:107708006173D20093453BD0821D5200D25E1112A4
:107718002274E022E173D200934531D0C21D520099
:10772800D25E1112A274802261741201934527D08F
:10773800020008325200D25E111222759022E174C2
:10774800120193451CD0020009325200D25E111278
:10775800A275A02261751201934511D002000A3268
:107768005200D25E11122276C022E1751201414602
:10777800934505D10B304400E35E1A124A768B76A6
:107788005A460523002A4BD1DFB27B1CDBB29C464C
:10779800791EBC1C89B2E4B22E4A464601239146A2
:1077A8002B4D307842405008134201D0684080B2D7
:1077B8004208034201D06A4092B25008134201D0F5
:1077C800684080B24208034201D06A4092B2500831
:1077D800134201D0684080B24208034201D06A4097
:1077E80092B25008134201D0684080B24208034266
:1077F80001D06A4092B2013989B201364945D0D1E7
:1078080043466146184DDA55120A5A54174B2A68EE
:107818009A4209D0220041462800FEF7F7FA1DE7F0
:1078280053465E00F31CAFE7012202211048FCF723
:1078380071FB220041462800FEF7E8FA0EE7042310
:1078480005249C4603270221A6E7C04678070020A6
:1078580001A0FFFFFFFF0000EE0400200605002046
:10786800F8070020EC0400206C03002000380140D9
:107878000004005070B5274B274C284A236080230A
:1078880020005B00264DA380A61DFF3B01784A40DF
:107898005108134201D0694089B24A080B4201D00D
:1078A8006A4092B25108134201D0694089B24A082D
:1078B8000B4201D06A4092B25108134201D069408C
:1078C80089B24A080B4201D06A4092B25108134269
:1078D80001D0694089B24A080B4201D06A4092B28D
:1078E80001308642D2D10F4DE2800F4B2A689A426E
:1078F80005D0082221002800FEF788FA70BD012271
:1079080002210A48FCF706FB082221002800FEF79E
:107918007DFAF3E7010310077C090020FFFF000050
:1079280001A0FFFF000400200038014000040050BF
:1079380070B5524B82B09A78022A01D002B070BD5D
:10794800DA781B791B0213435BBA1AB29CB2002A7D
:107958000FD04B48018809B29142EFD003806B46A3
:1079680012121A7101A9022200205C71FFF726FB8E
:10797800E4E7444C444B2600236080231B01A3808A
:107988001023A3713E4B20009A89404D12B2121267
:10799800E2719A8917362272DA8912B21212627269
:1079A800DA89A2721A8A12B21212E2721A8A22733F
:1079B8005A8A12B2121262735A8AA2735A8912B27E
:1079C8001212E2735A8922749A8A12B212126274DB
:1079D8009A8AA274DA8A12B21212E274DA8A2275C8
:1079E8001A881B8812B2A375012312126275284ADD
:1079F80001784A405108134201D0694089B24A08C7
:107A08000B4201D06A4092B25108134201D069403A
:107A180089B24A080B4201D06A4092B25108134217
:107A280001D0694089B24A080B4201D06A4092B23B
:107A38005108134201D0694089B24A080B4201D06B
:107A48006A4092B201308642D2D1124DE275120AD2
:107A58002276114B2A689A4205D019222100280063
:107A6800FEF7D4F96AE7012202210C48FCF752FA22
:107A7800192221002800FEF7C9F95FE7FC08002059
:107A8800040500207C0900200110100001A0FFFF60
:107A9800FFFF0000000400200038014000040050EF
:107AA80010B5124B1B78002B06D0114B114A1B88BE
:107AB80011781BB2994210D00F4B1B78002B03D0C2
:107AC8000E4B1A78012A00D010BD5B78032B0AD020
:107AD800102BF9D1FFF7CEFEF6E75378032BEBD145
:107AE800FFF76AFDE8E7FFF723FFEDE7F808002056
:107AF80004050020780700207C0A0020FC080020EC
:107B08001020F0B55021C646604D614C2B6800B579
:107B18001A6882B002431A60196223681A6802431D
:107B28001A60196200F0CCF8FA215A4E3822C900BE
:107B38003000FFF749F9FFF793FA2800FEF73AFA01
:107B4800802255492800FEF7B9F92000FEF732FADD
:107B5800802252492000FEF7B1F99622504952007E
:107B68005048FBF787FE002202214F48FCF7D2F964
:107B78004E4B002098466423424601A953800222B6
:107B8800FFF75CFA00280BD16B4642469B885BBA2C
:107B9800138013881BB2013373D01388002B70D065
:107BA800FA210020490000F0A9F95021012000F035
:107BB800A5F90A21022000F0A1F93D4F3D4D3E4CA8
:107BC800002000F0B1F9002824D1012000F0ACF920
:107BD80000282CD1022000F0A7F900282ED12B78FC
:107BE800002B46D12378002BEAD0802100222E4892
:107BF8008900FCF78FF9FFF753FF802100232A48FB
:107C0800012289002370FCF785F9002000F08CF927
:107C18000028DAD03800FDF7E9FB80212248490026
:107C2800FCF77EF9012000F07FF90028D2D0FFF799
:107C380025FA022000F078F90028D0D03000FFF7AC
:107C4800DDF87379022BCAD11C49306BF8F708FCB0
:107C5800F8F7E8FE434600B2D8821849706BF8F787
:107C6800FFFBF8F7DFFE434600B298822B78002B23
:107C7800B8D0FFF715FF00232B702378002B9FD077
:107C8800B3E70123424613808AE7C0460004002078
:107C98006C03002098040020FC09002078080020CC
:107CA80020050020E8000020000400500405002002
:107CB800A00100207C0A0020F80800200000C8422B
:107CC800002225211B4B5A609A605A701A701A615B
:107CD8005A615A731A73DA611A625A761A769A6274
:107CE800DA625A5401395A540D315A639A635A5414
:107CF80001395A540D311A645A645A5401395A5484
:107D08000D31DA641A655A5401395A540D319A659D
:107D1800DA655A5401395A540D315A669A665A54DA
:107D280001395A540D311A675A675A5401395A544D
:107D38007047C046840A00206A4B1A68002A07D098
:107D48001A68013A1A60002A02D1674B01321A7088
:107D5800664B5A68002A0AD05A68013A5A60002AC3
:107D680005D101325A701A78012A00D19CE01A69AB
:107D7800002A0AD01A69013A1A61002A05D101328B
:107D88005A731A7B012A00D191E0DA69002A0AD0D5
:107D9800DA69013ADA61002A05D101325A761A7E87
:107DA800012A00D186E09A6A002A0CD09A6A013A20
:107DB8009A62002A07D1012125329954013A9A5C26
:107DC800012A00D179E05A6B002A0CD05A6B013A8B
:107DD8005A63002A07D1012131329954013A9A5C39
:107DE800012A00D16CE01A6C002A0BD01A6C013AF7
:107DF8001A64002A06D101213D329954013A9A5C4D
:107E0800012A60D0DA6C002A0BD0DA6C013ADA6405
:107E1800002A06D1012149329954013A9A5C012A73
:107E280054D09A6D002A0BD09A6D013A9A65002AAF
:107E380006D1012155329954013A9A5C012A48D059
:107E48005A6E002A0BD05A6E013A5A66002A06D199
:107E5800012161329954013A9A5C012A3CD01A6F87
:107E6800002A0BD01A6F013A1A67002A06D101219D
:107E78006D329954013A9A5C012A30D01C4B1A6829
:107E880001321A6019681B4A914201D100221A6016
:107E98000920002218490B780133DBB2984252417D
:107EA800524213400B7070479A685A605FE75A69EC
:107EB8001A616AE71A6ADA6175E7DA6A9A6282E72A
:107EC8009A6B5A638FE75A6C1A649BE71A6DDA64E7
:107ED800A7E7DA6D9A65B3E79A6E5A66BFE75A6FF5
:107EE8001A67CBE7000B0020FC0A0020840A002058
:107EF800800A0020FFFFFF7F7D0A002010B50928B7
:107F08000FD8012484F310884300064A1B189B00ED
:107F1800D0184160816000214170D45481F31088E9
:107F280010BDFEE7840A0020092808D8420012186C
:107F3800054B92009B185A78D0B2012A01D0002034
:107F4800704700225A70FBE7840A00200300821859
:107F5800934200D1704719700133F9E7014B186853
:107F68007047C0460C00002070B500260C4C0D4D23
:107F7800641BA410A64209D1002600F031F90A4C6E
:107F88000A4D641BA410A64205D170BDB300EB587E
:107F980098470136EEE7B300EB5898470136F2E709
:107FA800C8820008C8820008CC820008C88200087D
:107FB800002310B59A4200D110BDCC5CC4540133E3
:107FC800F8E7F8B504000D0000F022F822000600DA
:107FD8000F002B0020002900FAF792FB002813D18C
:107FE8000022002320002900F8F712FA00280BD0FD
:107FF800FFF7B4FF212300220360002310001900BB
:10800800F9F7D6F806000F0030003900F8BD000077
:10801800F0B50A000D006D4904000300080087B0A0
:108028002840884211D122002B0020002900F9F7AE
:1080380003FD02000B0020002900F8F755FD04009D
:108048000D002000290007B0F0BD002D11DC6900EB
:1080580049082143F5D00020854210D022002B008A
:1080680020002900F9F7B0FF02000B00F9F7A0F88B
:10807800E5E7281515D180240021640307E0DA0A12
:1080880015385B05002AFAD0F5E752000131224283
:10809800FBD04C1E001B20241D00641AE5408B40B9
:1080A8002A434B49120344188021120B49031143F8
:1080B800C00703D4DA0F490051185B00002562108D
:1080C800490080240592DA0F5218162029005B0017
:1080D800A4030E19964202DC3119921B2D19DE0FEA
:1080E8005200013892195B0064080028F1D120265B
:1080F8008027040004963F06C619B446914202DB65
:1081080014D19E4212D860466646C0190091002ECE
:1081180003DAC643F60F8E190096521A6345894151
:108128004942521A61465B1A0099E419DE0F52005F
:108138009219049E5B00013E7F080496002EDBD155
:108148001A431FD0234E244F306871683A687B6801
:10815800009201933268736802920393009A019B1C
:10816800F9F732FF02000B0002980399F8F75AF961
:10817800002807D0306871683A687B68671C0FD19F
:10818800049C0135154B6A10D2186308ED0702D517
:10819800802109060B4305991C0009058D1850E735
:1081A800F8F7A2FC7768366802000B003000390047
:1081B800F8F72EF9002804D0023463426341ED1821
:1081C800E0E7012301349C43DCE7C0460000F07F70
:1081D80001FCFFFF68000020600000200000E03F75
:1081E800F8B5C046F8BC08BC9E467047F8B5C0460E
:0881F800F8BC08BC9E4670476C
:10820000A012000892120008701200089C120008C8
:108210007012000886150008701200089C120008F1
:108220009212000892120008861500089C1200089D
:10823000581200085812000858120008F8150008D3
:10824000000000000000000000000000000000002E
:108250000100000002000000030000000400000014
:10826000000000000000000000000000000000000E
:1082700000000000000000000000000000000000FE
:1082800001000000020000000300000004000000E4
:1082900006000000070000000800000009000000C0
:1082A000010002000400060008000A000C00100093
:1082B00020004000800000010804020408010101C0
:0882C0000101010307010000A8
:0482C800E1000008C9
:0482CC00B9000008ED
:1082D0000024F40001000000040000001000002051
:1082E00000000000040B00206C0B0020D40B0020C9
:1082F000000000000000000000000000000000007E
:10830000000000000000000000000000000000006D
:10831000000000000000000000000000000000005D
:10832000000000000000000000000000000000004D
:1083300059F3F8C21F6EA501000000000000F03FD5
:0400000508003119A5
:00000001FF
